:10000000F01F0010313200002D3200002D320000B0
:100010002D3200002D3200002D32000000000000C3
:100020000000000000000000000000002D32000071
:100030002D320000000000002D320000B912000037
:1000400065100000651000006510000065100000DC
:1000500065100000651000006510000065100000CC
:1000600065100000651000006510000065100000BC
:1000700065100000293200002932000029320000FA
:100080007113000089130000A1130000B9130000D0
:1000900029320000991400002932000029320000A2
:1000A00029320000293200002932000029320000E4
:1000B00029320000293200002932000029320000D4
:1000C00008B500230B60036000F056FD08BD08B5BD
:1000D0000A20002101F0ECF808BD000038B50C4BF7
:1000E0000D1C041C19680B4803F0CCF8212103F007
:1000F000C9F8011C012001F08BF9012001F068F919
:10010000291C201C02F00EFC012001F071F938BD01
:1001100078800440001BB70008B50A4B0A481968EC
:1001200003F0B0F8212103F0ADF8011C012001F02B
:100130006FF9012001F04CF902F0D2FB012001F02F
:1001400057F908BD78800440001BB70013B596200E
:10015000000201F0DFF917480D210C2200F0ECFB42
:1001600000F02AFB14480021032200F059FC00F0A3
:100170002DFBFFF7D1FF114801F0C0FB002401F077
:1001800073FA002802D000F095FE00240A2001F046
:10019000BFF8684601A9FFF793FF009B002B03D12E
:1001A000074B01349C42EADDFFF7B6FF054801F03A
:1001B000A5FB13BD793600004C3400005B34000011
:1001C0006F1700006F34000073B518200021FFF78F
:1001D00085FF0024384E012001F00AF9374D98358B
:1001E000002C01D0002000E00620012101F060F881
:1001F000684601A9FFF764FF009B002B21D1002C6A
:10020000F0D12B68002B0DD02D4B00941A681132C1
:100210001A6004E002F00EFB009B01330093009B88
:10022000102BF7DD274BF618DED518200021FFF73D
:1002300055FF224B94331C6863425C4100F090FAF6
:10024000CEE7002C03D0182BC5D100F0C7FA009BD5
:10025000182B10D1019BC22B29D11B4B00221968EE
:1002600001311960022900D11A6001921FE0FFF7E5
:100270006DFF00230193154B1548196803F002F830
:10028000212102F0FFFF011C012001F0C1F8012033
:1002900001F09EF80098019902F044FB074B94335B
:1002A0001B68002B95D100F05BFA012492E7019BBB
:1002B000732BE0D1DBE7C04620BF020088040010AA
:1002C000C00200100CFEFFFF700100107880044097
:1002D000001BB70037B501F07FFB00F019FC00F000
:1002E0007DFA1E480D210C2200F026FB00F0EEFDE9
:1002F0001B4D1C48291C01F001FB3C2400F05CFA5A
:10030000A1B2281C032200F08BFB013C00F05EFA36
:10031000282000F0FDFF0A2CF0D102F0B1F90F23E4
:10032000009311481E231149114A02F065FA00207A
:100330000421012200F0E6FD0020021C042100F04F
:100340002FFE00200521012200F0DCFD0020052108
:10035000021C00F025FEFFF737FFC046793600008B
:10036000883400007A340000F5310000C10000003C
:10037000C002001000B500E001300378202BFBD054
:1003800000BD00B5031C303BDAB2092A01D8181CA5
:1003900008E020231843031C613B5738052B01D983
:1003A0000120404200BD70B50E1CFFF7E3FF0025A1
:1003B000041C06E0FFF7E5FF002805DB2D010543DF
:1003C000013420780028F5D13560201C70BD000074
:1003D00070B5054E051C0E24013C295D301C01F052
:1003E0008DFA002CF8D170BD9434000000B50E23B6
:1003F000013BC25C002A03D1002BF9D1012000E0AF
:10040000002000BDF8B500240E2700E0C02403231F
:100410001C4221D13E1C66432E4D7019FFF7E6FFAA
:10042000002815D0601C78434019FFF7DFFF002833
:100430000ED0301C1C304019FFF7D8FF002807D021
:100440002A367019FFF7D2FF002801D0043416E0D5
:100450002148211C01F052FA381C60431D4B013425
:10046000C018FFF7B5FF1D4801F048FA0C2C04D066
:100470001C2CCBD0502CC9D001E01024C7E7FF2C96
:10048000C5DD174801F03AFA164C201CFFF7A0FF13
:10049000154801F033FA201C0E30FFF799FF13487E
:1004A00001F02CFA201C1C30FFF792FF104801F0DD
:1004B00025FA201C2A30FFF78BFF0E4801F01EFAA8
:1004C000201C3830FFF784FF616D0B4801F016FAED
:1004D000F8BDC04624050010973400001C7D0000C4
:1004E000A034000088040010A6340000AC340000E2
:1004F000B2340000B8340000BE34000070B50E1CE9
:10050000FFF738FF0D25041C2078FFF73AFF00287D
:1005100007DB01347055013DF6D2201CFFF72AFF9E
:1005200000E0002070BD000073B5394D08682B78DD
:10053000002B06D1374801F0E1F902F0A1F80123C0
:1005400042E00378412B1BD1334C0230211CFFF7D2
:10055000D5FF002851D00378422B4ED1211C023008
:100560000E31FFF7CBFF002847D00378432B44D14F
:10057000211C02301C31FFF7C1FF002846D13CE0AE
:100580004D2B23D1254C0230211CFFF7B7FF00284B
:1005900033D003784E2B30D1211C02300E31FFF7BF
:1005A000ADFF002829D00378472B26D1023001A9BE
:1005B000FFF7F9FE019B002B1FDB2A3C63651848FF
:1005C000184901F09BF900232B701FE001A9FFF7E8
:1005D000EAFE0378202B01D0002B0ED1124E00240E
:1005E0000E250199611869438919FFF787FF0028D3
:1005F00003D00134042CF4D108E002F041F808489B
:100600000A4901F07BF9024B00221A7073BDC04603
:1006100098020010CA34000088040010B2040010D0
:10062000E4340000F934000024050010FC3400001C
:1006300073B54D68154E25E0281CFFF79BFE01A9F8
:10064000FFF7B1FE019B051C002B1BD0D8B2FF2B7E
:1006500009DD00F0FFF9041C01980012C0B200F09F
:10066000F9F9019003E000F0F5F9002401900199F7
:10067000002907D0301C221C01F040F90198211CF0
:10068000FFF72CFD2B78002BD6D173BD033500006E
:1006900008B5064A012113784B40137001D0044974
:1006A00000E00449044801F029F908BD7503001071
:1006B000143500001C3500002535000070B5051C00
:1006C00001200821021C00F06BFC072401260120F8
:1006D0000821002200F064FC2A1C22413240002044
:1006E000022100F05DFC01200821021C00F058FCF2
:1006F000013CECD270BD10B50021041C0A1C022084
:1007000000F04EFC201CFFF7D9FF10BDF7B5012308
:1007100000930023019372B66C46061C02AF01CC15
:1007200050235B421843C0B2FFF7E5FF0020FFF7FC
:10073000E2FF1020FFF7DFFFE020FFF7DCFF0025DE
:1007400002200021012200F02BFC705D0135FFF733
:10075000B5FF842DF4D18436BC42E0D162B6F7BD3A
:1007600008B5AC20FFF7C7FFAE20FFF7C4FFA520F8
:10077000FFF7C1FF08BD08B5AF20FFF7BCFFA420FD
:10078000FFF7B9FF08BD08B5AE20FFF7B4FF08BDFD
:1007900010B5041CF820FFF7AEFF201CFFF7ABFFDD
:1007A00010BD10B5041C8120FFF7A5FF3F2020409D
:1007B000FFF7A1FF10BD000008B584220248002108
:1007C000520001F0C8F808BD7D03001008B50248CA
:1007D000FFF79CFF08BDC0467D03001008B501204F
:1007E000021C082100F08EFB0120021C082100F0F1
:1007F000D7FB00200221012200F084FB002002210F
:10080000012200F0CDFB02200021012200F07AFB42
:1008100002200021012200F0C3FB02200621012258
:1008200000F070FB02200621012200F0B9FB03203A
:10083000011C012200F066FB0320011C012200F0D4
:10084000AFFB0320011C002200F0AAFB02200621BE
:10085000002200F0A5FB06210122022000F0A0FBEF
:10086000FFF7AAFFFFF7B2FFA220FFF744FFA02087
:10087000FFF741FFC020FFF73EFF0020FFF788FF92
:100880000A2000F045FD4020FFF735FF2C20FFF740
:1008900032FF322000F03CFD2E20FFF72CFF3220EB
:1008A00000F036FD2F20FFF726FF0A2000F030FD74
:1008B0002520FFF720FFAF20FFF71DFFA420FFF743
:1008C0001AFF0020FFF76DFF08BD000000B50F29DB
:1008D0000ED883280CD8CB08842253430722C01893
:1008E0001140044B80220A41111C1A5C1143195417
:1008F00000BDC0467D030010F0B55B18DBB216E00A
:100900008425CC086C4307270F40802504193D41FE
:10091000EFB2A6189C4605E0064BE5182B7801348B
:100920003B432B70B442F7DB01316346C9B29942B5
:10093000E6D3F0BD7D03001000B5084B1860084BEE
:100940001970084B20211A70074B1970074BD108FA
:100950001970500701D00131197000BD78030010E3
:100960008504001087040010860400107C0300102A
:10097000F0B5284B89B01B780024C01A264B06928C
:1009800005911B68221C04E002310C190132A4B24B
:10099000D2B2195D8242F7DB1B195B780391029397
:1009A00000222CE000994B4303999A198A4214DAE9
:1009B000194A0025126892191219D3189B780493CA
:1009C0000123049AAB40134204D07919C9B20798A5
:1009D000FFF77CFF0135082DF2D101360837F6B25A
:1009E000FFB206E00099059A069F8B18DBB200263D
:1009F00007930A490B789E42D4D3019A013201929F
:100A00006B461B79029900938B42EBD309B0081C0B
:100A1000F0BDC04686040010780300107C0300106F
:100A2000F7B5171C061C0D1C00F0B5FF80B2019035
:100A30000024FFB208E0305DE9B23A1CFFF798FFEE
:100A400001302D18ADB20134019AA3B29342F2D312
:100A5000F7BD000000B50F23020918408000031FF6
:100A600000D52833002B0EDB511E03208842804125
:100A70004042002807D1242B06DC04218A1A0349AE
:100A8000CB18985C00E0002000BDC0467C3A000016
:100A900010B5041C211C144800F0A6FA211C1348B0
:100AA00000F0A2FA211C124800F09EFA211C114805
:100AB00000F09AFA211C104800F096FA211C0F4809
:100AC00000F092FA211C0E4800F08EFA211C0D480D
:100AD00000F08AFA211C0C4800F086FA0B48211C11
:100AE00000F082FA10BDC04620400440244004407B
:100AF000284004402C400440384004403C4004401E
:100B00004040044044400440484004404C400440BD
:100B1000F8B51020FFF7BCFF094C271C14372578C7
:100B20006678281C311C002200F0ECF90234281CE5
:100B3000311C012200F034FABC42F0D1F8BDC046AD
:100B4000A43A0000F8B50B4C271C143725786678BA
:100B5000281C311C012200F0D5F90234281C311C5C
:100B6000002200F01DFABC42F0D10020FFF790FFF8
:100B7000F8BDC046A43A0000F0B589B00024049046
:100B80000591FFF7C5FF0220072101220694079473
:100B900000F0B8F902200721221C00F001FA201C05
:100BA0000B2100F0D3F9A04202D1182306930124AF
:100BB0000021264D03916A782F78111C0192381C70
:100BC000012200F09FF9381C0199002200F0E8F999
:100BD00003231F4E029314E03078717800F0B6F9C9
:100BE000002807D103991B4AA3008A5C1833694681
:100BF0005A500134029A039B013A01330292039343
:100C0000023EE30F00210122A2424B41DBB28B42A4
:100C100002D0029B8B42DFDA381C0199002200F0DF
:100C200071F90199381C012200F0BAF90A4902351C
:100C30008D42C0D1201E06D0069B049A05991360F0
:100C4000079B01200B6009B0F0BDC046A43A00002C
:100C50007A3A00007C3A0000B83A000000B50A4B2E
:100C600000211960094B01221A6019601A60196885
:100C70001142FCD0064B01221A60064B80221968F3
:100C800052020A431A6000BD708004407480044020
:100C9000788004408080044008B500F025F90C4BB2
:100CA00003201A68120B12031A600A4B1A68120BFF
:100CB00012031A60084B1A68120B12031A60074BD2
:100CC0001A68120B12031A60FFF7C8FF08BDC0466E
:100CD00000800050008001500080025000800350CE
:100CE00070B50F4C0F48211C00F008FE201C00F0CE
:100CF00005FE0D4E0D4D00242B196159DA68301C8C
:100D0000074B143400F0FAFD642CF5D1084800F0CC
:100D1000F5FD00F019FB011C064800F0EFFD70BD69
:100D2000163B0000B83A0000D13A00000000001065
:100D3000DC3A0000033B0000F0B53C4B8BB01D7863
:100D4000002D3AD03A4B02901B6801209B685DE071
:100D500001342378202BFBD0002B3AD0B30008338A
:100D60006A469C500136FF2D01D135E001342378CD
:100D7000202B01D0002BF9D1202B02D1002323708E
:100D80000134012E1BD12A4F2A4B06223B600192CF
:100D90003D1C09E02B680298196800F00FFE00283E
:100DA00008D02B6814332B60019B013B0193002B6F
:100DB000F0D132E03B681D7901E0041C2E1C237841
:100DC000002B06D000230722B2425B41DBB2002B8E
:100DD000BFD1002E1CD000E00025154C022E05D1FD
:100DE0000398154900F0EAFD002801D0AE420AD868
:100DF00023681248D96800F081FD236810481969FA
:100E000000F07CFD04E02368F0B29B6802A99847DB
:100E1000064B1B78002B07D103E00198011CFFF75C
:100E20005FFF084800F06AFD0BB0F0BD98020010AB
:100E3000A002001000000010103B0000123B000058
:100E4000F4340000193B000038B5041C154D0A2885
:100E500008D002D808281CD110E00D2802D07F2825
:100E600017D10BE02B6800221A700F4800F046FDE6
:100E70000E4C201CFFF760FF2C6012E02A680B4B21
:100E80009A420ED90A48211C00F038FD2B68013B1C
:100E900006E00748211C00F031FD2B681C7001336F
:100EA0002B6038BD9C020010163B0000980100101A
:100EB000253B000008B503E000F0B4FBFFF7C4FFDA
:100EC00000F0D2FB0028F7D108BD000008B5034AA6
:100ED000034B04481A6000F011FD08BD9801001092
:100EE0009C020010193B0000044B40211A680A4381
:100EF0001A60034B01221A707047C046808004407C
:100F0000A402001070B50E4B061C1B780D1C141C9F
:100F1000002B01D1FFF7E8FF013E022E03D8094B59
:100F2000B600F35800E0084B1A68012C03D1AC401E
:100F300014431C6003E00124AC40A2431A6070BD5E
:100F4000A4020010903B00000080005038B50F4B09
:100F5000051C1B780C1C002B01D1FFF7C5FF0020DE
:100F6000032D11D8281C012302F082F9020406087F
:100F7000074A04E0074A02E0074A00E0074A10680F
:100F8000A3401840431E984138BDC046A40200103B
:100F9000FC3F0050FC3F0150FC3F0250FC3F03501F
:100FA00070B50E4B061C1B780D1C141C002B01D1B8
:100FB000FFF79AFF013E022E03D8094BB600F35803
:100FC00000E0084B1A68012C03D1AC4014431C60AC
:100FD00003E00124AC40A2431A6070BDA4020010DB
:100FE0009C3B0000FC3F005038B5084B041C1B78AC
:100FF0000D1C002B01D1FFF777FF236818229343C4
:10100000236023681D43256038BDC046A40200103C
:101010001F234209184001238340181C014B9200F2
:10102000D050704700E100E0054B3F221A60054BAD
:1010300001221A60044B40211A688A431A607047E3
:1010400024800440D88004403882044008B5044B12
:1010500040211A688A431A60FFF7E6FF08BDC046C0
:101060003882044008B50320FFF7F8FD094B012240
:1010700052421A60084A1268002A00D01A60074BD0
:101080001A6801321A60064A00231360054A136089
:10109000C04608BD088204400C820440A80200102B
:1010A00004C000403CC0004008B5FFF74BFD0A48B3
:1010B0000021FFF799FF09480021FFF795FF084835
:1010C0000021FFF791FF07480021FFF78DFF064839
:1010D0000021FFF789FF08BD08400440004004409C
:1010E000AC400440144004401C400440F7B501905B
:1010F000FFF7DAFF574B01991A68574B1A6000291E
:1011000001D0564B00E0564B564A04211360564B13
:10111000564C1A68564D0A431A60019A002A54D058
:10112000544B0027544E1F60544B301C1F60391C19
:10113000FFF75AFF381C09213A1CFFF7E3FE381C61
:1011400009213A1CFFF72CFF4D4B80221968032020
:1011500011431960336807218B43336033680221E0
:101160000B43019933604B005B1899015B1801999F
:101170009B005B1843490B60434B1968014319609E
:10118000424B4349186801401960196809200A4315
:101190001A60FFF73DFF226880239B001A432260FC
:1011A00001213C4A494211602A68324913432B60AD
:1011B000394B02221A60394B01221A601F601A60F3
:1011C00018681042FCD001230B600720FFF720FFB6
:1011D0000820FFF71DFF0A20FFF71AFF0C20FFF77A
:1011E00017FF0B20FFF714FF23688022934323602F
:1011F00022682B4B1340236022682A4B1340236044
:101200002268294B134023602268284B1340236037
:10121000019B002B03D101221E4B52421A602B6806
:10122000802213432B602A6880235B0013432B60CA
:101230002A688023DB0013432B602A6880235B012C
:1012400013432B602A6880231B0113432B6030BF9C
:10125000F7BDC0463882044034820440BF18000005
:10126000FF1800003082044010ED00E000820440CE
:101270000482044004C00040644004400440014033
:101280008080044018C0004014C000403CC00040B2
:101290000FF0FFFF08820440708004407480044017
:1012A000FFFEFFFFFFFBFFFFFFEFFFFFFFF7FFFF6B
:1012B00008B5FFF71BFF08BD00B5064B1A680132E1
:1012C0001A601B68013303D1034B1A6801321A609C
:1012D00000BDC046B0020010AC02001000B5074BC4
:1012E00098420AD8064A00231360064A0138106063
:1012F000054A1360054B07221A6000BDFFFFFF007F
:10130000B002001014E000E018E000E010E000E09F
:1013100000B50C4A1368002800D10120C1438B425C
:1013200004D809E011688142FCD301E0591C081877
:1013300011689942F6D203E01168C91A8142FBD3C1
:1013400000BDC046B002001010B5064BFA21186867
:10135000054B89001C6801F095FF044B5C43201885
:1013600010BDC046B0020010AC0200103789410029
:10137000034B01221A60034B1A6801321A6070474E
:1013800000C00040B4020010034B01221A60034B5E
:101390001A6801321A60704700000140B80200105C
:1013A000034B01221A60034B1A6801321A6070471E
:1013B00000400140BC020010034B01221A60034BA5
:1013C0001A6801321A60704700800140C0020010A4
:1013D00000B5002803D1044B01221A6003E0012864
:1013E00001D1024B186000BD04400140048001405F
:1013F00000B5002802D1044B186004E0012802D196
:10140000024B00221A6000BD0440014004800140EC
:1014100010B5041C002906D1164B96201968C0008F
:1014200001F030FF011C002C0FD1134B80221868F3
:10143000920002431A60114B03221C60104B19608A
:10144000104B1A608022D20211E0012C11D10A4BFC
:1014500080221868D20002431A600B4B00221A60E7
:101460000A4B032219600A4B1A6080221203094BAF
:101470001A6010BD7880044080800440BC020010D7
:101480001840014014400140C00200101880014083
:101490001480014000E100E008B5184B1A680E23E3
:1014A0001340062B0DD1164B9E221B68DBB2134254
:1014B00004D0144A5360144B1B681EE0D9071CD596
:1014C00001E0042B05D1104B1868C0B200F0BBF846
:1014D00013E00C2B06D10B4B8022596852000A43B3
:1014E0005A600AE0022B08D1054B1A68054B910699
:1014F00001D5002200E001229A6008BD088000406A
:1015000014800040C4020010008000400048704772
:10151000C402001070B52B4C2B4B80229203DA676B
:1015200000219022061C201C00F015FA0023A36065
:1015300000F072F8254B07251A68254CAA431A605B
:101540001968012211431960224B1968A9431960D7
:10155000196811431960204B802118684901014323
:1015600019601E4B1E481A608322226019681D4BA9
:101570001B68584301F086FE311C000901F082FE11
:101580001949030A194A0B60C0B203231060236093
:10159000174B1D60174B186860201C680440602CB6
:1015A000FBD101E0146800E001201C680442F9D17D
:1015B000044B01221A70104B802292031A600523FB
:1015C0000B6070BDC402001004E100E0A4400440C0
:1015D0000C800040A8400440808004409880044073
:1015E000001BB70078800440048000400080004069
:1015F000088000401480004000E100E000B5044A8B
:10160000202311681942FCD0024B186000BDC0466F
:10161000148000400080004008B5FFF777FF0023EA
:10162000437308BD08B5FFF771FFC27B031C821826
:10163000107CDA7B7F2101320A40DA735A7B013A4F
:10164000D2B25A7308BD10B5041CFFF75FFF837B4D
:101650007F22C3181C74837B013313408373437B45
:101660000133DBB2437310BD08B5FFF74FFF407B7A
:10167000431E984108BD30B5002402E005700134D6
:1016800001301D5D002DF9D1121B131C02E0017009
:10169000013B0130002BFADCD043C0170240A018F8
:1016A00030BDF8B5051C0F1C1E1C541E092B01D89B
:1016B00000240FE0181C0A2101F0E4FD221C031C89
:1016C000391C281CFFF7EDFF041C2D1805E02F70B6
:1016D00001340135013A002AF9DC301C0A2101F0FD
:1016E00015FE30312970601CF8BDF8B50C1CD917F7
:1016F0005F18061C4F40551E092F12D9381C0A21AD
:10170000002B03DA01F0BEFD434202E001F0BAFD16
:10171000031C211C2A1C301CFFF7E7FF041C351892
:1017200013E0002B00DA951E002201E0B4540132D0
:10173000A91A0029FADCEC43E4172C403519002BD8
:1017400003DA2D232B7001340135381C0A2101F0F6
:10175000DDFD30312970601CF8BD73B5069E041C98
:101760001D1C3009531E00280AD000901A1C201C92
:101770002B1CFFF7F2FF241805E021700130013423
:10178000013A002AF9DC0F231E40092E01D8303619
:1017900004E0002D01D0373600E0573626700130C6
:1017A00076BDF0B585B0041C0F1C002801D00021C7
:1017B000017000256BE0252903D02170013201342E
:1017C00005E05178252904D1217002320134013518
:1017D0005DE0302903D001320292202101E0023283
:1017E0000292029E9C4632782D3A50424241B618EF
:1017F0000296002205E00A235A438218303AD2B2F8
:1018000001363078031C303B092BF4D90296AE1810
:101810006346BE4201D97A1BD2B269280ED006D8DF
:1018200063282CD0642809D058283ED119E07528A7
:101830000AD078280FD0732837D11AE01E1D201C3B
:101840001B68FFF752FF04E01E1D201C1B68FFF7FA
:1018500028FF331C17E01E1D1B68201C009300236B
:1018600004E01E1D1B68201C00930123FFF775FF79
:10187000EFE71E1D201C1B68FFF7FDFEE9E71A6855
:10188000012022700433029A241801322D18117895
:10189000BD4201D200298ED10023BD4201D2237066
:1018A00005E0013C2370013D01E001256D4205B0DA
:1018B000281CF0BD10B50C1C131C6421221CFFF762
:1018C00070FF10BD30B5A3B0041C0D1C24220A49C2
:1018D00019A800F01EF86846211C2A1CFFF7EAFF31
:1018E000632803DD19A800F097F8FEE7684600F0CA
:1018F00093F823B030BDC046A83B00000FB407B535
:1019000004A901C90191FFF7DDFF03B008BC04B0D1
:10191000184770B50323041C184205D10D1C041C84
:10192000194201D1934201D3002311E0131C40CD91
:10193000043B40C4032BFAD8141FA4080134A400AC
:10194000032309191A400419EEE7CD5CE55401336D
:101950009342FAD170BD30B50B040D061D430D4303
:101960000B021D430323041C93420DD218420BD1DA
:10197000131C043B20C4032BFBD8141FA408013400
:10198000A40003231A400419002301E0E1540133A9
:101990009342FBD130BD00B5002300E00133C25CAF
:1019A000002AFBD1181C00BD00B5031C01E0013169
:1019B00001330A781A70002AF9D100BD00B502E09F
:1019C0000130002B06D00A78037801319342F7D01A
:1019D000981A00E0181C00BD08B5FFF75DF90B4828
:1019E000FFF77CFCFFF780FAFFF730FB9620000240
:1019F000FFF790FDFEF7F2FEFEF7DEFE044A054813
:101A0000111CFFF77BFFFFF761FA08BDE02E000015
:101A1000163B0000CC3B000010B5041C02E0013472
:101A2000FFF7ECFD20780028F9D110BD00B50B4B75
:101A3000984201DD0A4BC0180A4A8310D35C032286
:101A40000240082152008A1A93401A1CC0239B00AE
:101A50001A40054B1B5C101C184300BDFF1700000B
:101A600000F8FFFFFA3B0000FA47000070B5C24CD7
:101A7000C248E26E416A531E9A41C14E1C2386B091
:101A80000B406D46F35817352A709F460C260323EA
:101A9000C66049111F2930D8BA4A89005258974662
:101AA0000D260D23F4E7636E16339B00E3581E1CCE
:101AB000EEE702260023EBE7636E16339B00E65841
:101AC0000023E5E70D260023E2E7A36DE66DB342B0
:101AD000DEDD0D26DCE702260223D9E701222A708B
:101AE000226E1021002A0CD1A74A0291101C00215D
:101AF0000096019501F028F82A7806B00120E266E8
:101B000070BD0A21F0E7321C9F48191C01F0A0F8B3
:101B10002A78F2E7321C9D48191C01F099F82A78BE
:101B2000EBE7321C201C191C01F092F82A78E4E73C
:101B3000211C1A1C1C31201C331C009501F06EF86E
:101B40002A78DAE70095201C1A1C0021331C01F0CA
:101B500065F82A78D1E7226E1021002A00D00A21E8
:101B6000221C0E3202910020211C0096019500F0EB
:101B7000EBFF2A78C1E7226E1021002A00D00A214B
:101B8000221C1C32EEE700957F48DDE700957F4878
:101B9000DAE7216E01222A701022002900D00A22E1
:101BA00079490292081C00220096019500F0CCFFB2
:101BB0002A78A2E7226E1020002A00D00A20724A5A
:101BC0000290111C101C1C390096019500F0BCFFFE
:101BD0002A7892E7216E01222A701022002900D073
:101BE0000A2269490292081C00220096019500F021
:101BF0007DFF2A7881E7226E1020002A00D00A207B
:101C0000614A0290111C101C1C390096019500F0CD
:101C10006DFF2A7871E7226E1021002A00D00A2178
:101C2000594A0291101C111C0096019500F05EFFAC
:101C30002A7862E7226E1021002A00D00A21221C95
:101C40001C320291201C211C0096019500F07CFFA3
:101C50002A7852E7216E01222A701022002900D032
:101C60000A220292201C0022211C0096019500F0FD
:101C70006BFF2A7841E7226E1021002A00D00A214A
:101C8000221C0E32DDE7216E01222A70102200296B
:101C900000D00A220292201C0022211C00960195ED
:101CA00000F024FF2A7828E7226E1021002A00D0B5
:101CB0000A21221C1C320291201C211C0096019535
:101CC00000F014FF2A7818E7226E1021002A00D0B5
:101CD0000A21221C0E32EEE7E018011CF31A5A1CEE
:101CE0001C31FFF716FE2A7807E728481A1C011C4A
:101CF0000E31331C00F0F0FE2A78FEE6E018E11801
:101D0000F31A5A1C1C300E31FFF703FE2A78F4E652
:101D1000211C1C311A1C201C331C00F0DDFE2A780B
:101D2000EBE6E018E118F31A5A1C0E30FFF7F1FD4C
:101D30002A78E2E6211C0E31ECE7E018F31A1C3099
:101D4000591C01F04FFB2A78D7E6E018F31A0E3041
:101D5000591C01F047FB2A78CFE6E018F31A591C0A
:101D600001F040FB2A78C8E6321C201C191C00F048
:101D700081FF2A78C1E6C0468804001024130010B1
:101D8000FC7700001C780000A404001096040010EA
:101D9000F8B5144C8C2560590130FFF747FE124B03
:101DA000A16E012298625E6A0240914201D0022037
:101DB000F8BD82070BD48822A15865590F1C1E3725
:101DC0000235BF003D51013103252940A150FF22BA
:101DD000920010408001B6108C220643A6500122CA
:101DE0009A60E4E7880400102413001070B50B49D2
:101DF0000B4A4B6A8C20DC051658A40E980500D5BA
:101E0000403C956E9B10012003409D4203D1341944
:101E10008C23D4508860012070BDC046241300106C
:101E20008804001030B50C4B20241D5D21241C5D5E
:101E30002D0124022C43DD7F882299582C43222532
:101E40005D5D081C2D031E302C438000C450013101
:101E500003200140995030BD8804001010B50B4993
:101E600088228B580320013B03408B501E339B007C
:101E70005A580C1C0B1C1C3320340F20011C114021
:101E8000197001331211A342F8D110BD880400105B
:101E900008B5144B1B68002B00D09847124A1369F1
:101EA000002B1DDD012B0DD00321181C8843591E6A
:101EB00000280AD00D4B0120D866116190215B5893
:101EC000136208BD9169002902D1591E074BF4E73E
:101ED00000239361054B01205161D8660F21ECE787
:101EE000024BEBE754030010241300108804001089
:101EF00030B50B1C093B012B00D930BD0023084D28
:101F000002E001330E2BF8D0EA18147FC25C944231
:101F1000F7D0044B08391A6811431960EDE7C04641
:101F2000880400102413001000B5082902D01929D4
:101F300007D000BD00230022C25401330E2BFBD179
:101F4000F7E742780823134203D00022027043705F
:101F5000EFE70F23037007234370EAE770B50C4CDB
:101F6000666F002802D00F239E430643F500094BFD
:101F7000AD1B6D00ED18281C311CFFF7D5FF0023A9
:101F8000E95CE218013311770E2BF9D1666770BD59
:101F9000880400102405001070B50F4C0F23666FE5
:101FA0009E4306436667082E14D0F500AD1B231C24
:101FB0009C336D00ED18281C311CFFF799FF00239E
:101FC000E218127FEA5401330E2BF9D1281C311C80
:101FD000FFF7AAFF70BDC0468804001038B50C4C4E
:101FE000616F082913D0CD006D1A231C9C336D003E
:101FF000ED18281CFFF77CFF0023E218127FEA543B
:1020000001330E2BF9D1616F281CFFF78DFF38BD0E
:102010008804001010B50D4C2023E05C2123E35C04
:1020200000011B021843E37F18432223E35C1B03D8
:102030001843FFF7FBFC0F231A1C02402277021102
:10204000134000126377A07710BDC04688040010CB
:1020500000B5094B5A6E16329200D2580D2A07D09D
:102060009A18507F117F0001021C0A435A6500BD77
:1020700029229A5C5A65FAE78804001010B5084BCB
:102080000F245A6E596D16329200D2580C4098188F
:10209000013204770D2A02DC9A180911117710BD5C
:1020A0008804001030B50F4B5A6E586D16329200EE
:1020B0009A58511C0D2A10D05C18247F9D182D7F32
:1020C00024012C435C650F249A18044014770D29D1
:1020D00002DC5B180011187730BD29241C5D5C659B
:1020E000F1E7C0468804001008B503480E22011C21
:1020F0001C39FFF70EFC08BDC004001008B50348EA
:102100000E22011C1C31FFF704FC08BDA4040010C2
:1021100008B504480022011C1C310D2300F0DCFC32
:1021200008BDC046A404001008B503480E22011CD7
:102130000E39FFF7EEFB08BDB204001008B50348E6
:102140000E22011C0E31FFF7E4FB08BDA4040010B1
:1021500008B504480022011C0E310D2300F0BCFC20
:1021600008BDC046A404001070B5174B0322002020
:1021700099184631097840000843013AF8D2197F8E
:10218000002201269C18351C0D4046340132257072
:102190004910042AF6D118770722002099184631F1
:1021A00009784000013A0843032AF7D1597F0422F5
:1021B00001269C18351C0D4046340132257049100B
:1021C000082AF6D1587770BD8804001000B50B4A74
:1021D00003230021D0184630007849000143013B19
:1021E000F8D2117707230021D01846300078490033
:1021F000013B0143032BF7D1517700BD8804001048
:1022000030B50C4900230A7F0125C8182C1C144046
:102210004630013304705210042BF6D14A7F012559
:10222000C8182C1C14404630013304705210082B7F
:10223000F6D130BD8804001010B5094C8C23E0584D
:102240000130FFF7F3FB074B98620F231A1C024083
:1022500022770211134000126377A07710BDC046A9
:10226000880400102413001010B5084C0E21201C07
:1022700001F0B8F8201C0E300E2101F0B3F8201C3C
:102280001C300E2101F0AEF810BDC04688040010CD
:1022900010B50C4C201C231C0E301A7F19780A43F1
:1022A0001A7701338342F8D1A36E002B03D0064B7B
:1022B000DB680D2B00D010BD237F2922A35463734C
:1022C000F9E7C046880400102413001010B50C4C28
:1022D000201C231C0E30197F1A780A401A7701330C
:1022E0008342F8D1A36E002B03D0064BDB680D2B85
:1022F00000D010BD237F2922A3546373F9E7C046A1
:10230000880400102413001070B50E4A84B0002316
:102310000D2500241118097F01306E46F154C10FBC
:10232000854261414942013308400E2BF2D100231E
:102330006C46E05CD118013308770E2BF8D104B05D
:1023400070BDC0468804001038B5A94A0F24506AF1
:10235000A84D83101C40A400A7492C598011095690
:10236000A746F82B02D9012040420BE0A3499B006D
:10237000CB589F460029F4DBA14B0120591840316E
:1023800000238B7138BD0029EBDB9D4B01205918D0
:10239000403101238B71F5E70029E2DB984B0120E6
:1023A000591840318A79DA66ECE7954B5A6E163245
:1023B0009200D1585C1801392077D15001200029B2
:1023C000E0DA0D21D150DDE70029CADB8C4B01207A
:1023D0005A6E16329200D258891A4A424A41DA6637
:1023E000D0E70029BDDB864B01205A6E16329200E1
:1023F000D150C7E7FFF7D0FD0120C3E7FFF7AEFDDF
:102400000120BFE70029ACDB081CFFF77DFF01209E
:10241000B8E77B4B88201958032401392140195013
:102420001E318900C8588C21585001239360012027
:10243000A8E7734B01205A6E16329200D158013131
:10244000D1500E299ED10021D1509BE7FFF720FDEE
:10245000012097E7FFF73AFF012093E7FFF784FE9B
:1024600001208FE7664B01205A6E16329200D15838
:102470000139D150002900DB84E7A2E7FFF7E8FD2E
:1024800001207FE75E4A01219823D150012079E79E
:102490005B4B00225A66012074E7FFF7EFFD012035
:1024A00070E7FFF721FE01206CE7554B00218C20DF
:1024B000195088201950196701239360012061E7A2
:1024C000FFF73CFE01205DE7FFF7ACFC012059E778
:1024D000FFF72AFE012055E7FFF7AEFE022051E785
:1024E000FFF716FE01204DE7454B01225A660120F9
:1024F00048E7FFF7D7FD012044E7FFF7FFFD012084
:1025000040E73F4B0120996E002900D03AE788242C
:10251000195903250139294019511E318900CC5818
:102520008C215C5090602DE7FFF750FE012029E7D9
:10253000FFF7AEFE012025E7314B0120996E0029FF
:1025400000D11FE7E3E7FFF75BFE01201AE7FFF783
:1025500061FD012016E72A4A9423D0580121414009
:10256000D15001200EE7FFF739FD01200AE7244B87
:10257000002294215A5098215A50012002E7204B02
:1025800001221A660120FDE61D4B0120597F9A7F2A
:10259000090112020A43197F0A435A67F2E6184BEF
:1025A00000221A660120EDE613690120002B00DCF1
:1025B000E8E65269124B0F211140D9771211202100
:1025C0005A54DFE6FFF7C4FD0120DBE6FFF746FCC7
:1025D0000120D7E6FFF748FE0120D3E6094B002291
:1025E000191C0E311A7001338B42FBD10120C9E650
:1025F000241300109C780000C07C0000DC780000F0
:1026000088040010CE04001038B5164C8C23E05816
:10261000FFF70CFAE36E9022134DA158A366002336
:10262000E3660131AB6003236862A15018400228C1
:1026300015D0032810D001280BD0FFF785FE002805
:1026400006DDAB68002B03D18C23E2581218E25050
:1026500038BDFFF79DFBF2E7FFF7C8FBEFE7FFF799
:1026600005FAECE78804001024130010034B012244
:10267000DA660F229A775A771A7770478804001023
:1026800010B5064C0649201C00F0ACFE0123E366A1
:102690000F23A3776377237710BDC046880400100B
:1026A0009C0E000000B5074B00201B680F2B08D1C3
:1026B000054B1A78824204D11868044B1840431E17
:1026C000984100BD640000108804001000FFFF0066
:1026D00038B5164B1A1C98321268002A04D0144BD5
:1026E0001D6801231D4001E094331D68114C63688F
:1026F0009D4202D12268002A16D0002D02D1002B63
:102700000AD111E00C4B1B68002B02D02168281C59
:1027100098470023236006E0074B1B68002B02D07C
:10272000281C291C9847656038BDC04688040010E5
:1027300070030010241300106803001013B5002369
:1027400000930193244B1B68002B02D0684601A91B
:1027500098472249009B0878214A00280CD0002B7A
:1027600002D00223137035E01378013BDBB2137003
:10277000002B2FD10B7009E0002B0CD11378002B0C
:1027800028D0013BDBB21370002B23D1154A136014
:10279000154A13601EE014490968581A4442604102
:1027A0004000107011480469021C002C04D08B42B8
:1027B00002D1102303610DE000290BD1102111611A
:1027C000019953619161084A1360064B0222196016
:1027D000034B1A7013BDC0465C0300107403001055
:1027E0006003001054130010501300102413001045
:1027F00008B5FFF7A3FF08BD10B5074C20600748D8
:10280000016007490A60074A1360074B029A1A6081
:10281000064A074B1A6010BD680300105C030010E5
:10282000640300105803001064000010F12700003A
:102830005403001008B5084B084A196812688A1A30
:102840001A6006D5FA2252001A60054B1A68013246
:102850001A60FFF73DFF08BD680000105803001024
:1028600070030010F7B50E1C0E21051C019200F03C
:10287000B9FD1A4B03240C279E420FDD09236B730D
:1028800001232B7328E0301C0A2100F09FFD301C2F
:1028900029550A2100F044FD0134061C002E06D003
:1028A000E30F0022A7425341DBB29342EBD1019ADE
:1028B000A31A033B2B70621B2B1C01E0195D59739B
:1028C000013BD1180229F9D10F231C1B002301E081
:1028D000013C2B55032CFBDCF7BDC046FFC99A3BDE
:1028E00038B50C4B01221A700B4B02221A700B4D9B
:1028F0000B4C08E01868884208D01B682360FFF77B
:1029000099FFFFF71BFF2B682168024A1078002807
:10291000F0D138BD74030010600300106403001090
:102920006C030010F8B52A4C051C60612948A161B0
:10293000031C94331B68002B12D1182D06D1C32918
:1029400004D138300E21162200F0AEF86369182B3E
:1029500004D1A369332B01D100F048F8FFF786FEBC
:1029600010231C4E23611C4F012333678C36FFF765
:102970004BFE3368BB4207D0184A93420CD1184B28
:102980001B680F2B08D103E0154B1B68102B03D1DC
:10299000FFF79EFEFDF79BFB124B1A68124B106867
:1029A0001968884205D012681A60FFF743FFFFF7E5
:1029B000C5FE084C236F002BD9D1FFF789FE182DD7
:1029C00003D094342368002B01D0FFF789FFF8BDB2
:1029D00024130010880400106A0C0000790D000018
:1029E00064000010640300106C03001070B5294CE3
:1029F00023681D68FFF774FF23681A689542FCD0AE
:102A00001E68FFF733FE244B1022244C1A61182253
:102A10005A6115229A61231C903300221A60FFF735
:102A200025FE0123236764361A4C1D4D0AE0FFF78B
:102A3000EBFD23682A681968914203D01B682B605C
:102A4000FFF7F8FE23681B689E42F0D1134D182053
:102A50002B1C903300211C68FFF764FF1820002115
:102A6000FFF760FF18200021FFF75CFF0D4B6000AF
:102A70001968001900F054FC3835011C0422281C88
:102A8000FFF7F0FE044B18225A610022201C9A61C5
:102A900070BDC046640300102413001088040010A9
:102AA0006C03001058030010F0B501390127002A0B
:102AB00011DD05780B1E0BDB3D4000E0351CC45CCE
:102AC0003E1C2640ED0064082C43C454013BF5D263
:102AD000013A002AEDDCF0BD30B504E0845C8D5C89
:102AE00085548C5401329342F8DA30BDF0B5474634
:102AF00080B4069CA446079CA04608AC27784446B0
:102B00002578002A1CD063450CDCCE5CD45C3419DB
:102B100064190025A74201DCE41B0125C4540133DC
:102B20009C45F2DA43461D7004BC9046F0BDCA5C79
:102B300052190025974201DCD21B0125C2540133F2
:102B40009C45F4DAEEE7C046F0B5474680B4079CF2
:102B5000069FA04608AC24784546A4462C78002859
:102B60002AD000291ED0002A47D0BB4204DD10E045
:102B7000C55401339F420CDBCE5CD55C751B2D1B0D
:102B80000024002DF4DA6544C554013301249F422A
:102B9000F2DA43461C7004BC9046F0BD00210024CC
:102BA000C15401339F42F4DBD15C49420C1BF5D088
:102BB0006444E1B20124F3E7002912D0002A19D0BD
:102BC000BB42E6DCCD5CD05C0133281A041BE40F69
:102BD0009F42F7DADDE7D15C013349420C1B611EED
:102BE0008C419F42F7DAD4E7CA5C0133141B0134ED
:102BF000624254419F42F7DACBE76546013DBB4252
:102C000004DDC6E7C25401339F42C2DBCA5C121B1B
:102C10000024561CF6D12A1C0124F3E770B5049E4B
:102C20000124347000290ED09A4203DD0DE00132F8
:102C300093420ADB855C8C5CA542F8D070BD815C58
:102C40000029FBD101329342F9DA00233370F5E712
:102C500030B50C1C91420ADA43185D7801341D70BE
:102C600001339442F9D14B1CC94364181C19002349
:102C7000035530BD70B5141C8A420ADD561E8319F7
:102C80001D78013C5D70013B8C42F9D10134A41ADE
:102C900034190023035570BDF0B5114B1A785B78D9
:102CA000825C1A4000D040220E4C0F49231C261C87
:102CB00004C32C3600221A6001240A1C1231177832
:102CC0005578C75D3D4202D01F6827431F6002321E
:102CD00064008A42F3D10433B342EBD10020F0BD4B
:102CE00061010010E8140010AD00001030B512238F
:102CF0004B43334A0131D3188A0051181A785C7853
:102D0000825C144204D02F4A5F245218947054708D
:102D10009A78DC78825C144204D02A4A7C245218C7
:102D2000533214701A795C79825C144204D0254ABB
:102D30007C245218A33214709A79DC79825C144294
:102D400007D0204C5F226418251CA235A1342A70BC
:102D500022701A7A5C7A825C144204D0194A7C246C
:102D60005218A03214709A7ADC7A825C144204D031
:102D7000144A7C245218503214701A7B5C7B825C9B
:102D8000144207D00F4C5F226418251C5235513471
:102D90002A7022709A7BDC7B825C144204D0094A40
:102DA0002E245218A43214701A7C5B7C825C13426D
:102DB00004D0044B5918F43127230B70002030BD88
:102DC000AD00001058130010F8B52D4C071C00255D
:102DD000201C20214F22FEF7BEFD002D04D0221C16
:102DE0007C23393223701370231C4F3300210135AB
:102DF00019705034052DEBD1214B2D22181C383081
:102E00000270181C37300270A1209A705A7040006E
:102E10005F221A541B481A54A320400019541A491F
:102E200008784978385C014204D0191C5331523378
:102E30000A701A700024211C381C0134FFF756FF59
:102E40000A2CF8D1114D124E00242B786A78FB5CC5
:102E50001A4201D0315905E03059FEF79CFD0D4969
:102E6000091A0A310C48043400F0C6FA0235242C41
:102E7000EBD10A49084800F0BFFA0520F8BDC0466A
:102E80005813001041010000610100106C00001097
:102E9000800000106301001098140010D07C000026
:102EA000F0B585B001900027FDF786FCB34C3E1CC1
:102EB000B34A7542754113687D19012B05D1B1489C
:102EC0000D210C22FDF738FD02E0002B00D1BEE001
:102ED000002303AA537023687F210B405B2B62D031
:102EE00028DC382B00D18BE013DC072B65D006DC07
:102EF000022B00D190E0062B00D0A8E03EE0212B71
:102F000000D181E0232B00D184E01C2B00D09EE077
:102F10007EE0402B64D005DC392B67D03F2B00D0FE
:102F200095E05BE0502B6FD0542B73D04F2B00D02B
:102F30008DE03AE0712B5FD00FDC622B68D005DCAE
:102F40005C2B63D05E2B00D081E051E06D2B30D044
:102F50006F2B36D0662B7AD129E0792B4AD006DC4C
:102F6000762B4BD0772B3DD0732B70D14AE07D2B45
:102F700021D07F2B23D07C2B69D135E031231370F6
:102F8000022E4BDD231C083B1B681940542908D036
:102F9000032E43D0231C0C3B1A687F231340542B71
:102FA0003CD14C2217E0322337E0332335E0342381
:102FB00033E0352331E036232FE037232DE038236B
:102FC0002BE039231370062E28DD231F1B681940C0
:102FD000232923D1472203AB1A701FE030231CE0C2
:102FE0002D231AE0412318E0422316E0432314E086
:102FF000442312E0452310E046230EE048230CE072
:103000004C230AE0502308E0522306E04F2304E05B
:10301000552302E04E2300E049231370ADB203A80C
:10302000291C0022FDF7FCFC23681A0605D5E91DC2
:1030300089B255480022FDF7F3FC2368DA0567D50D
:103040000735A9B251480022FDF7EAFC60E0236889
:103050000122134206D0A818C0B200210722022381
:10306000FDF74AFC23680222134205D0A81DC0B216
:1030700000210623FDF740FC236804210B4205D004
:10308000A81DC0B202220623FDF736FC23680821E2
:103090000B4205D0681CC0B207220223FDF72CFCAE
:1030A0002368DA0606D5681CC0B204210222062372
:1030B000FDF722FC23689A0606D5681CC0B20021E1
:1030C00002220623FDF718FC23685A0606D5681C61
:1030D000C0B2042107220223FDF70EFC23681A0662
:1030E00007D5281C09300222C0B20821131CFDF7A5
:1030F00003FC2368DA050BD5EDB2281C0930C0B2F9
:103100000B210A35FDF7E2FBE8B20A21FDF7DEFBF1
:10311000013604340C370B2E00D0C9E61C480321BD
:103120000622FDF709FC1B4D1B4E1C4F0024019A83
:103130002B78D35C6A781A4205D0A3009859395D80
:103140000922FDF76DFC01340235092CEFD1FFF7A0
:10315000A9FA002827D006240321201C00F0E0F85B
:103160000321C5B2201C00F031F9281CC9B2FDF7BB
:10317000ADFB092C14D10B24EEE7C046E814001077
:103180007001001079360000513B0000D87C00002F
:10319000343500006C00001074010010A400001011
:1031A00001340E2CD8DDFDF711FB05B0F0BDC04693
:1031B00070B5041CFFF770FD201CFFF771FE0A4B71
:1031C0001B78002B0ED0201CFFF7FEFD074CC823F8
:1031D0005B00074EE518211C301C5034FEF78EFBB7
:1031E000AC42F8D1002070BD7503001058130010D8
:1031F000F434000008B5002805D0FDF7BCFA0748F4
:10320000FFF7D6FF08E0FDF7BEFA054B1B78002B51
:1032100002D00448FEF772FB08BDC046A2050010AC
:1032200075030010DA7C000000B5FEE700B5FEE78C
:1032300008B50A4B0A4A0B4903E0107801321870AE
:1032400001338B42F9D3084B0849002201E01A7080
:1032500001338B42FBD3FDF73DF8FEE70000001081
:10326000337D000098010010980100101415001023
:1032700002B4714649084900095C49008E4402BC09
:103280007047C046002934D00123002210B4884280
:103290002CD301242407A14204D2814202D2090185
:1032A0001B01F8E7E400A14204D2814202D24900A6
:1032B0005B00F8E7884201D3401A1A434C08A04249
:1032C00002D3001B5C0822438C08A04202D3001BDF
:1032D0009C082243CC08A04202D3001BDC082243F6
:1032E000002803D01B0901D00909E3E7101C10BC1A
:1032F0007047002801D00020C04307B4024802A153
:103300004018029003BDC046D90000000029F0D04B
:1033100003B5FFF7B9FF0EBC4243891A1847C046F0
:10332000002941D010B4041C4C40A44601230022C3
:10333000002900D54942002800D5404288422CD3BC
:1033400001242407A14204D2814202D209011B01B7
:10335000F8E7E400A14204D2814202D249005B00B6
:10336000F8E7884201D3401A1A434C08A04202D31E
:10337000001B5C0822438C08A04202D3001B9C085F
:103380002243CC08A04202D3001BDC0822430028C1
:1033900003D01B0901D00909E3E7101C6446002C87
:1033A00000D5404210BC7047002806D003DB002047
:1033B000C043400801E08020000607B4024802A193
:1033C0004018029003BDC046190000000029EBD050
:1033D00003B5FFF7A7FF0EBC4243891A1847C04642
:1033E0007047C04600B5002905D00023013903709D
:1033F00001300029FAD100BDF8B5041CA30719D18A
:10340000231C04CB0F4D104E50199043021C201C5E
:1034100032420FD1181C0B4F04CBD51995433542BE
:1034200008D1181C074F04CBD51995433542F1D06C
:1034300000E001300378002BFBD1FEF7B5FA201C29
:10344000F8BDC046FFFEFEFE808080805345524995
:10345000414C20434F4E534F4C4500444D20313595
:103460004343204D31422072656164790D0A000D9D
:103470000A4279652E2E2E0D0A0052504E204341ED
:103480004C432025730A0D00444D20313543432021
:103490004D3142002578000D0A2530327820200079
:1034A0000D0A413A20002020423A20002020433AD1
:1034B00020000D0A4D3A200020204E3A2000202006
:1034C000473A20253032780D0A0057616974696ED9
:1034D0006720666F722074686520646174612E2EA7
:1034E0002E0D0A0043616C63207374617465207251
:1034F0006561642025730D0A004F4B004641494C1D
:103500004544006B65793A202530327820253032E9
:10351000780D0A00656E61626C65640064697361B0
:10352000626C6564004C43442064656275672025C5
:10353000730D0A0003030000000303005C00030393
:103540000C000C03037C287C03037C447C030324D1
:10355000104803032854080303000C0003033844F5
:10356000000303443800030320100803031038103D
:103570000303804000030310101003030040000306
:103580000320100803033844380303007C000303BE
:10359000645448030344542803031C107C03034C65
:1035A00054240303385420030304740C03032854E5
:1035B000280303085438030300500003038050001D
:1035C0000303102844030328282803034428100376
:1035D000030454080303384C5C0303781478030392
:1035E0007C5428030338444403037C443803037C9D
:1035F000544403037C1404030338443403037C1051
:103600007C0303007C00030320403C03037C106C1C
:1036100003037C404003037C087C03037C047C039D
:10362000037C447C03037C140803033844780303BD
:103630007C146803034854240303047C0403037CC0
:10364000407C03033C403C03037C207C03036C1060
:103650006C03031C601C030364544C03037C440090
:1036600003030810200303447C0003030804080339
:1036700003808080030304080000070804000000A2
:1036800000BF01BF01090500000700070007000790
:10369000130A00002000E400FC003F00E700FC00EB
:1036A0003F002700040F0800000C011E01FF03FF6C
:1036B000032201E201C2190D00000E001F001101DA
:1036C0009101FF007E00FC00FE0113011101F001D9
:1036D000E0140A0000EE00FF0111011101BF01EE2C
:1036E00000E00130011001050300000F000F0A0582
:1036F0000000F800FE03070701040B0600000000AD
:1037000001040707FE03F80F08000000000A000E7E
:10371000001F001F000E000A110900001000100019
:103720001000FE00FE001000100010080400000051
:1037300004800780030D0700001000100010001027
:1037400000100010080400000000800180010D0737
:10375000000C000FC003F0003C000F00030F080036
:1037600000FE00FF01010101010101FF01FE10083F
:103770000000000002010201FF01FF010001000141
:10378000100800008601C7016101210131011F01FC
:103790000E010F08000082008301110111011101C7
:1037A000FF01EE11090000300038002C002600FF58
:1037B00001FF012000200F08000080009F011F0171
:1037C00011011101F101E10F080000FC00FE010BE5
:1037D0000109010901F901F00F08000001000100D1
:1037E000C101F1013D000F00030F080000EE00FFD2
:1037F00001110111011101FF01EE0F0800001E006F
:103800003F0121012101A101FF007E080400000009
:10381000008C018C010804000000048C078C03124A
:10382000090000200070005000D80088008C0104BE
:103830000104011109000048004800480048004800
:1038400000480048004811090000040104018C01EF
:103850008800D80050007000200D0700000200030F
:1038600000B101B9010F0006190D0000F800FC01BC
:103870000603FB06FD0505050505FD05FF0506011B
:10388000FC01F8120900008001F0017C004F004F9C
:10389000007C00F00180010F080000FF01FF011112
:1038A0000111011F01FE01E0110900007C00FE0072
:1038B000830101010101010183018211090000FF5F
:1038C00001FF010101010101018301FE007C1008DB
:1038D0000000FF01FF01110111011101110111018E
:1038E0000F080000FF01FF0111001100110011007D
:1038F00001120900007C00FE008301010121012169
:1039000001E301E20112090000FF01FF01100010B4
:103910000010001000FF01FF010A0500000101FF77
:1039200001FF0101010B060001000101010101FF7E
:1039300001FF10080000FF01FF0138006C00C60005
:103940008301010110080000FF01FF0100010001D7
:10395000000100010001160B0000FF01FF010F0034
:103960003C00F000F0003C000F00FF01FF011209D5
:103970000000FF01FF010F001C007000E001FF01CB
:10398000FF01130A00007C00FE0083010101010118
:1039900001018301FE007C0F080000FF01FF0121EF
:1039A00000210021003F001E140A00007C00FE00E0
:1039B00083010101010101038307FE047C04120954
:1039C0000000FF01FF01210021007100DF008E01D6
:1039D0000001110900008E009F0111011101110168
:1039E0001101F301E211090000010001000100FFD3
:1039F00001FF010100010001110900007F00FF002B
:103A00008001000100018001FF007F110900000713
:103A1000001F007800E001E00178001F0007190D89
:103A200000000F007F00F001E0017C001F001F007C
:103A30007C00E001F0017F000F120900008301C744
:103A4000016C00380038006C00C7018301110900C7
:103A500000010007001E00F801F8011E0007000128
:103A6000120900008101C1016101310119010D013B
:103A70000701030100070008000A010018111013D4
:103A80003831303378717073C8C1C0C38881808386
:103A900084848782C5C4C7C275747772353437325F
:103AA000151417120207020802010003010903049A
:103AB0000204020503050006436F6D6D616E64200C
:103AC0002020204465736372697074696F6E25737A
:103AD00000252D3130732025732573000D0A54798C
:103AE000706520273C636F6D6D616E642D6E616D36
:103AF000653E203F2720666F7220706172616D7392
:103B00000D0A00557074696D65202575730D0A00E6
:103B10003F0025730D0A0D0A00564F594147455283
:103B2000203E3E200025630048656C70004E6F20EB
:103B3000706172616D73004B65792070726573738B
:103B4000003C6B6579313E203C6B6579323E202E1E
:103B50002E2E0044756D70206D656D6F7279006C4E
:103B6000004C6F6164206D656D6F72790074005454
:103B70006F67676C6520646973706C6179206F751D
:103B80007470757420746F20636F6E736F6C650052
:103B9000008001500080025000800350FC3F015023
:103BA000FC3F0250FC3F0350737464696F2E633A0C
:103BB00020696E637265617365204D41585F53548F
:103BC00052494E475F53495A450D0A0025735479AF
:103BD000706520273F2720666F722061206C697313
:103BE00074206F6620617661696C61626C65206328
:103BF0006F6D6D616E6473257300A106C105557507
:103C000020C5F0A0B04E453502DC312B1017134F04
:103C10009CC300E302044A116A596686E294CF10FD
:103C20000CB0065A0482F00020C24A00DE1DE22ECB
:103C30000277590555B5414D4999918A0872958485
:103C4000035555654753256A41C99A1076043101D9
:103C5000C0C0B40F44F080544599599D8821323535
:103C6000880B04820310D5DE4012150066C4333081
:103C700009401904508050508E5024A46A0021201D
:103C80008A400156552521218490D1646346A216AD
:103C9000D8A410602254423044744A881115146923
:103CA0005520B8072678100846002C06885C0909BC
:103CB0000200000000000000000000100300808CE3
:103CC0000831212310C14110130011D025D8C74459
:103CD0003121B2B7A061BB987363501021FB40261D
:103CE0001185204852911088580100848802303193
:103CF000006288CE3C0044511444898988B8BBAA2C
:103D0000AB2B1221003233232213757700C0CC4431
:103D10004566B9BB45B4BBB888894030885DF83387
:103D200033D1467844EC0010519D2ED1552522A266
:103D300000019099D9DDFDFFFF03C1088C302148B7
:103D4000844C0001D34C4802D8940CBEF240B0C45D
:103D50003C0C8A37120E59DF049DF14D100EE423FE
:103D60003F001232135011FB0C088CC0400101AC13
:103D70001336C804599D531659DFDF1C76B3CCB8EF
:103D8000D30E8803018410D071A1885335D2ED5031
:103D9000F04404C900D160F3E24E0C4A2703250128
:103DA000130973390CD8FDDD335D7C13163923CA32
:103DB0002710102520560C8C443B5114318413D00D
:103DC0000E6BBCC784EC3A120729C400C433281711
:103DD000188010C9442D63E022084548D1FC0D3FEE
:103DE000C8FF480F0C0C0C0044328C7D1001A1243C
:103DF000170F481DF2760924B70FAA0A2010AA0A45
:103E0000109340230011A4884C70CC12A31C05729F
:103E1000801DFEC45CDC4518D4F9001B13855B28AB
:103E2000843F0F0CC62C41CC473C414C473FA66D0C
:103E30004B1B102F49515A1C17731041C700B0611A
:103E40003E1D5A1444FC813136463D48C00C513069
:103E50001180C41C08C22183CC0C313311D15060B5
:103E6000B13E4721840C4C14F1CC0F03CD70046794
:103E70003192BBCB3300282333F100B3C600044892
:103E8000C010222B1F6A33EDC1A8C118033450049F
:103E90008282A2A00710462466369F04351789A0A7
:103EA000D42C3EFD7E008F8D7D3113CA30623C4C98
:103EB00084E020B654F184F640282EED35431500F9
:103EC00044E2C86114F111D507D04F4C37200730B8
:103ED000C9F1BC348BD29E615020AC547685D1029E
:103EE0004BD80D4D043348814C11CC481014C15CA3
:103EF000684C43A141D98C7B0F0091301A0743389D
:103F0000404C4F0800C03040A802C04444C1540493
:103F10000133F9471138453188EC041210000000D4
:103F2000310424044C9381C00C0000300210024381
:103F3000147140084C0C02C0880C7037A80900208E
:103F400031032C0012302348088423210386101AE1
:103F5000E28A47C8A800E160A06E08205020C8404F
:103F60002420C84000C68C008DC08884204A4C089C
:103F70002182000220444004C4930220A008325849
:103F8000E54110BF741D48F4841C9C0320A584A047
:103F9000FC3D3008C0D280C4F4432C82A812B11179
:103FA0000641F4A1636C72890820134212B00140EB
:103FB000088042408AE4937F24CD03178282C31C89
:103FC000F2FB000C140C0460631800311048140755
:103FD0001002044A8A01D336D8BD138C080182A08E
:103FE00028CB00100B2050428155CF838DDDFB3351
:103FF000000B0000804064F9BE26C107034CD80DB9
:1040000001825550D14FFC0452F1074515407C0008
:1040100011014442BD43CB4008820C08820C083297
:10402000500CE00021002120412204C4F958D8C4DA
:10403000D304118D4D464CD30E91AA0CA004AE387A
:10404000BF87B807FF378E8B2C71C7D9B80F1447BD
:10405000082E8A0720FF424FED4700360104E38C0B
:104060004310F4760BA2788CB349480012626017B3
:104070003B020018B248B84354085400E25E199459
:104080002C719B0103648816638295D544422135C7
:1040900003A4041D6014072029D0D90A803020E22F
:1040A000FE42A518880009680A0045A22461C029BB
:1040B00035728C5F2016640F31045DEBEE95F20CC7
:1040C0003FA73510E24C431041C8C3BC34D330295C
:1040D000F140E6F823124EC4713D379F2BF77A1357
:1040E000AD1BC4103FA85606A2FCA090D2C61FEF7D
:1040F0004F450200550031088002228403484432B3
:1041000030A38BC2A24B88C0000EB0359381408E85
:104110004C041601C18D6098418E04862806D0C4D7
:104120004C040A312302028130117200098612B355
:10413000C774C403309530C021F0123031C12F5EF6
:10414000002241B1105402C5805412317280EC9C9F
:104150008328CD0432D2C8C858CA4852858C60859D
:104160008C24858C60C55032125429236225234843
:104170009532B25621C830A2C4C4521005445155DC
:1041800011114A5554554985085E12445544451449
:104190009415554554557454D1552195CBC40510EB
:1041A000C509C13009022042204CE18E8EAB4F2060
:1041B00010B9E4C6FFFF4D1763CA00F2299D301401
:1041C0008F5111A036120412D0E54948507AE47795
:1041D000086109EA440D2060A03E80820A2205148D
:1041E0003C445F0414420445421253806541404CF4
:1041F0004C0462C82120C4A841F2061A15102015EB
:10420000051455104CCC540140A02C2E400C0059E4
:10421000260413310E101333527446300A04013150
:10422000120C44440082C08CE0133130003232263C
:104230008C4081000281840231003144000144003D
:10424000000011D388C80018480404008824C0C4A2
:104250000484342EE2A2C82227C004310A3013207D
:104260008404083044D0CC144D044CC8C484444267
:10427000C320F020201004451005110F00229C0CD3
:1042800001004C9301C3C0091688C01012323010CF
:104290001220444C1854804505985008E300850CC2
:1042A00012822404000481080D2010201088448408
:1042B0000048301186844012001133338D60800233
:1042C0000B291180213111500404CC002413D0009B
:1042D0003333A12CA1921A0D05D040390903F28481
:1042E000901C4D22820DCC30D0941C068AC82C6BB9
:1042F000C3F7C01CA3F079B0820010C848E88880DA
:10430000C212108035C40810115D0205A423804438
:10431000804091C23BE3400D02208010048E0820B3
:10432000F33C0F1104897BC35C00310010205070F6
:1043300020E8104CA3024E86D6101D384C8301068F
:1043400075CBA63C309EA218B0C9F318C8A030A403
:1043500020133138D3915890043D8A67802003E1BF
:10436000345D0C1434104810B4807319D49130D3D8
:104370001441180B10871C3210618C3912104C0339
:104380002110142412417DC86C18C6D4DD10121AF5
:1043900037305E22F15C08353D62563C08A2483851
:1043A0000788D825C619CF15B01D152386E08620AD
:1043B00031473104D120903F00008A0B4A50B28827
:1043C0000150C74462197210C0D8239EC4332C6DAB
:1043D0000F2A584C3C330411CB87A925A184D5144E
:1043E000303E12469852837AAD1C076845A062821F
:1043F000C0303838180130070C00DC043D55320F4E
:1044000093A104D69716020EC88C848012238BB217
:1044100082B0AC47420C8DC02410C63346052149FA
:104420004812928484C9639049364899492360119F
:10443000B684C260B904650F00216433360182E19D
:10444000144F114098B3DD4BD66A4110C33F1C8412
:104450005C1C43711CC771F12161EFA11D0F3BC0B2
:10446000323C3F31CCF21CFF073B0A9CE01078093C
:10447000CE3B82CE7F0412892028D6230D3418C368
:104480004C2033033C4C38474C118470C70B00045C
:10449000111151440EF0088C2050FC1189F1445444
:1044A000344D4D2C0131F4D33490D0E984818150C6
:1044B000F30F024020A3C81F42E48030F33439399F
:1044C0001981B3DC0C0183C840D3E424E132C8FC79
:1044D0004B4C39F18001600981028A0D13010A28D1
:1044E00076F8A000FBF4BF6183BF10106288E3413F
:1044F0000317AE4610DAF33DC7C4400400A14CCC0C
:10450000494851C1120104040F218402224A48146F
:1045100035104000E30048CCA8C8E844084440A453
:10452000043A20110312C478084424080021110021
:104530000061125112481810200112A44540009247
:10454000B24C0C100E1081000010211011A3442158
:1045500060100B2A23B22BA2400A502800110884B5
:10456000028440940C408C00231630023112308AB1
:10457000040E318A440C00A07AA30E4E1C11418413
:104580004430140E53DD124FC411C3C44F102745DD
:10459000C7F43C06AB33314371B8C3A03A9FC16442
:1045A00010B31BE318443162A82D974CC81148C4BE
:1045B00008034062CC021D1A682023C655618B8A0D
:1045C00038CD92820CC620D4C43436B2C4053540EE
:1045D0000912880A3FE23BF5124C4577C794E9F689
:1045E0000C458084A210C85096FB202185C5EA2F77
:1045F0001280003B7074091490009582060410200C
:10460000440030004070281403500841449841038E
:104610004020020C01B123CF49330C0311F14704B0
:104620000D180319D260931803B1AA03408D070433
:1046300073047DE300D0041110D316911431D1100E
:10464000C30010640460000CC0C0000444BE645089
:10465000D086983B314414330001C83001813311B6
:104660008D99049D91D38C4DE444A42C2431225186
:1046700011E51F00310D441E533D144021600862B6
:10468000583644144913219C2C11B04C22238064C9
:104690009F0CA1D2594C4CB9409574540C22183B34
:1046A0001085DB208A0F14430418308CE840809179
:1046B00001490183040C1C43884C11FBA118B0393B
:1046C000099D363F7240030E31404B1253E0904437
:1046D0003E4D044140D065B218F4134352D5E38FE8
:1046E0008499DB14A6044C282B638C28211C1ECC37
:1046F000C523885C7AD5A1C1CEC8013CA0000C04BA
:104700003F3CD74040C4144A00F0448004031A8A56
:10471000C348F101D5044404A2A4306B4564884425
:1047200011C10061C0E10013C11786023012274792
:1047300010A144CD298113A3024433340A8402001A
:10474000012C6C50A1C7D74344C82412A082C3C512
:10475000F1FC7F32FCC4E8F24444300001CC4C0050
:10476000109052531C9D004390614CFC8131188184
:10477000250C84E0C4AB03315900008110440007CC
:10478000C4344B847D158E048034112211090882B3
:1047900010224E00130C828807190E3407583D1062
:1047A000110B037F100B651405F30F4C4E041842D8
:1047B0000A5D0FF2AAD88B930821F5E28698C9D436
:1047C0004074BAB274A4364D72601D19494FCFF4CB
:1047D00087F04C4C44401841045828180441883A4A
:1047E000DFBDBD7B1FFF3112868E0A023EC0C8218D
:1047F00055882088EA1C3B000000CF4E7038EE0F31
:1048000041A0210C6E0484A50200BCFB3279401348
:10481000CE35244E203C063018E06500666071AC51
:10482000E0A94E4E5C2650E0006FB4EFDF7823071E
:104830008BEBC241A06500668784210C3D4C0404CB
:10484000448465003075666330176673301266CD38
:104850005A3014665B2666CF883D4CB95C8CEF1CE1
:10486000E0207314FB8100C360003B02E07724D09A
:1048700043ECC9DC101EF81EE83357CA06751B4509
:104880000E12B84E20305ABC70E0E0D59C619C33CB
:104890000ED9A0D99C01401B04044419A410A8847B
:1048A00004446EE59C6E0CE5370CDD37048CA923BF
:1048B00049BCA9A8854E480940134429E176FCFD6E
:1048C00000EDAD1C621C629CC906CC4714B7D4B77E
:1048D000543794B90ACC7FB67F6666CCEB666666C1
:1048E00099A8B61CCB666694C7CC9399A8B6B69C1B
:1048F000A2E202DCC83366CC47D433CC231CD08D73
:104900000ACC3F142BCC5D0B5C66666666CC479484
:104910003714654F81A86666666666666666666673
:10492000CC9754B7540B56E33010C6B3CC37E3CC16
:10493000DB666699A8B6B69CC833CC8F947B99A8E1
:104940001CC8BB66E6438C079467545714479443CE
:10495000CC2F2BDC2B5C444C47E616B6DCD4EB8624
:10496000A6445459229D2EE01CEAA04884854E6638
:10497000666666F8FC941FD43754279417541F14A6
:104980000F1433F6D3D016D3F667CC63E6167676DB
:104990008648845C53CCB35C23CC3F1C85A8C4718F
:1049A000061CE399A82399A8669C6666668BCCA72B
:1049B00094AF99A8C8E3CC4FF846E8941D1F911E08
:1049C00099A89C83CC659F945F8C31A7542B71ACC4
:1049D0001D529C710ACC3F99A8B65C236699A85CCD
:1049E0007D0699A8B61CC87506CC410794CF99A836
:1049F00066665CF502CC450794319F5BCC69232B3E
:104A000014A7CCFF5403CCF3065CC906142BCC6767
:104A1000610ACC4F73148BCC17666681A8DC1366D1
:104A20006666666666666666CC3F941F5C231C13EA
:104A30009C85A87D06141BCCAFCCA79477239457F4
:104A400014E714AFD48FCCA59F94B3CCA31C9016BD
:104A50005394B714BF1433661CC47906141BCCA33B
:104A6000541FD497CC950A6B66661C89066699A874
:104A70001C7506663366CC271C621CC106F8FCF662
:104A800063D0164B3030066666CC1766305046C48D
:104A9000C3666666666681A89C91061C1010E64691
:104AA00046B63C02C49906CC6F9449076699A81C87
:104AB0008D06CC519F94859F99A8C8A3CC27C894F4
:104AC00093DC73CC5714431C62629CC4C82B9CC4F7
:104AD00044C4854E133373C38382C27232121030C2
:104AE00070C08087C7773717113171C18184C47452
:104AF0003414183878C88884C57535157140D54088
:104B0000C14CF5A871400E882B7140B0AECDAC857C
:104B100038C9ACBE5541F1404938A188C1AC8D3887
:104B20006140DD40C14CB14C8C6055A4AE28714051
:104B3000C5404938A14C7940D540C14C65448DAC45
:104B400038E03051A6A64E70F866A030049C58306C
:104B500009063008A5A86DA4DC50D09050D4EB68AD
:104B6000C4C44E9C90A8A0706E1C5090D0654EDCC2
:104B700050D4F34CA0EEE04E70F83CE6BCE8E58083
:104B8000B9A028E6F62B9A26E3FA46BEBA0E666866
:104B90009C0AED4CB9A0A8F14CFA1F4E224C17BE4E
:104BA000AE38FD40280E78BE1EFD40AEF83C567073
:104BB000AEF04E70B80E384C4FEB0E330EAE1B3DC0
:104BC000ACB940BEA74EEEA70C834C7701BC0E4893
:104BD00021BE0E1B0EAEB940FEF59C81024EEED7F3
:104BE0000CD34CC743000000000000BC88E4E8D8A8
:104BF000787CA8FCF844404CF474DC48A5363D327F
:104C0000B896913387349D26DCA3DBA4DDA5B39150
:104C1000B9928993DD149115A0FB1A48333663319C
:104C20004A169533B5348C26D5A3D6A4D7A5A3911F
:104C3000B792BB93B5943B95D8FB8300E201EA029F
:104C40002003BBD3BCD4BAD59821713177308940C9
:104C50003E30743110320649BEFFC300E601EB025C
:104C60002A031ED3EED4FFD5ED07EF08F1098A40E1
:104C70003244002006108549B04C7719AC580C2BF3
:104C800021BC4EF04E7098E05819A4E28BBB9DC039
:104C90009AB085A04D908649D8E000484936353510
:104CA00033442B251B3408200B490021005200629D
:104CB00047754274323053435843401638268F2389
:104CC000B623E804F405FF060C070E081009471682
:104CD00069160B100A2066040E050D066C4077302D
:104CE0007B2080106B4075307A207E10CCD8DAC2E1
:104CF000C0E3CBDCDBC3E40CD18059A40C21BD2183
:104D00008C7D8AF510813CF0CD8CA18839880C7996
:104D10008F654421AC1532F51061406588704D40B7
:104D2000653C630EF3818CE32E0E7AFE4B48CC3348
:104D3000CC23C488445CA606E669174687CECE23FA
:104D40005C62EE4F4C0761A00EA6AEBB4CA13F0DBE
:104D50003C818C46936ECE5C5A5E26E6433ED4542C
:104D6000D3EEE116D84E3ECE6BAED8221ED8AEAEF4
:104D7000BEEB1E2EAE8ECE93D83ED86EEED454B37C
:104D8000EED93C6ED8469C7D14EE132E62F38E4213
:104D9000FAF3DCA34CBB794079407940A188854087
:104DA0004938D14C213C1EA606E655166D16DC6628
:104DB00054EB5EFD38CC3BBEBE11A00D408C2B11D8
:104DC000A00D404C8766660011A08D3C8C3F4E5C68
:104DD00066508D384C1BBE1EE0EE4E6E5E546F94D6
:104DE000E7D41F5447145F9CD09CE0DC9090109057
:104DF0005090105030165CE09094F36B1CF9149CAA
:104E0000505C109CE05CF9149C50DCE05CF9145C94
:104E1000E01CF9141CE0C8481B0EBAFE43884C1B6A
:104E2000CC13485EEECE5AF6137AFA4CF78C2BAEC2
:104E30000ECECE4E5C1050EE6AFA2F6A1B2A8EEE12
:104E400058EEEEEECEEEFA9F8EFB2EEE66DB4EEEC9
:104E500098EE4C1B8ECEEE8E5B2EEE98EE4C0BE653
:104E6000F7EEEBCC5FC84C37487361A0A3444BC44A
:104E70004CAB8C1B841388036E8E00818C3B26F612
:104E8000278EB32E6600FD384C5F98EE6600853C99
:104E900011A09538D8AE0E263B6EEE3BD454AF260B
:104EA000E36E4E7D14EE133E8EF32ED4CEEE54A35D
:104EB000D88E8E4E5C50D89C90905B8A8ABEEB1E3A
:104EC000D8AE4E2ED88E1E62ABAEFAAEFA737E66A8
:104ED0001E8E9B98CCB7CCA30D3C8B5ED8AE98AE03
:104EE000CC1FCC1F866EDA73D8C13C4C4B7940FD89
:104EF00084CC3F0D3C4CA0BEE0B058468C213C8C8D
:104F00000D3DA1882938CCA1898CF1CDA188653CC3
:104F10004CA0BEF1CF4E5C7A360E8E4CA0730801C9
:104F2000A48C33F59C15CCBBE6E784EEBB9CE22356
:104F3000C1CC9BE1A01EBED05CA20645543D4CDD19
:104F400036B1A801A408059C8C1F888415CC9B2829
:104F500005A84E7038B1A85E5AF643880656BC665E
:104F6000B6CEEE0DA406781CEA4B6A4F1C908C1747
:104F70003616C12EF99C8CF99D5658F59C06567034
:104F8000381E1AEEB61C23DCDC7CB6E316EE7CCAB7
:104F9000CA8C43D497DCDC7CCACA6E0EEE0E7C1C35
:104FA0008C1B1C7CEEC3C2D4C2AEFC1CEAEECE7CD1
:104FB000AE1C5BA6AE0E70387C8C137CEAF0986653
:104FC0009F91CC84491E8C6BED80B9A060E6235C78
:104FD000154E7C0630089C6217484E3613EEA2F33D
:104FE00069A4B8AEE0CA0A0ACAEAEA4A8C330E06D5
:104FF0000E46E04ACAEAEFE00000505D707D909DE9
:105000003D3E1E2EC8019248F50E515E717E919E66
:105010004D4E9D9E79CC8C4BB8E633A646A8A5A8EC
:105020008102ADAEB1A801A4E1A01EBED05CA2E693
:105030006365CC8C236D202B886D2084068CE10366
:1050400045543D4CE065CC0C15A00ED8AE8CBD038C
:105050008C551FB1A8608444064E701C56792330CD
:10506000FA621F069F30A806BF62CB30B0C6161C7E
:10507000108ECAEABC30063A308C152F0C33D88C0F
:10508000798FD84E3096BC704E1C1006BC70CE6224
:10509000E21B380EB0A0E08CDD2FE6E69D3A006200
:1050A0001F024B3030063B8C052A30B0CB30500607
:1050B0002B48C38816300A9C022730B24B3070064A
:1050C00033764830AC1B1C62DB4E1CD01006BC3063
:1050D00096069C021388566376BBC9B830301C0A0A
:1050E0003F16E202138430C203764B5C6262C8430F
:1050F000765B1CA2304006174830D85B762330DA46
:105100002B763B30E24899B85A5E861686064646AC
:105110001C10068C912BBC30064E1C1046309BBCDC
:10512000704EA6BC6E70B04CA04425BA4E1C100246
:10513000D09006BC305AA03DACBC705394F981F0BD
:1051400023F910AECCA07039B8CCF59C0B21B8AEC9
:10515000619E21B859A478EE5670EE0924619C8BAB
:105160000924AE6D02C89940CCD76544F0B0ABC8F5
:10517000AEB940ABC855388BAEC8613C63B0B1B86E
:105180004613A64E300979A83B9C4EA22805A84E8E
:1051900070388C539C222233998C548DD758A0B0F0
:1051A000FA63EE59A4FA3BB1B86EAEB1B8B9A8EB48
:1051B0008C53300E9C629F998C540779AC8E652479
:1051C000EE3C066524F5A8EEE0F91049A4FC1C0AA3
:1051D0003C6ACA1681CC605E7CFAA0265CE260FC68
:1051E00046E0311C704C2BCDA80813A88102311C5D
:1051F000AE00B04CBB0405A8A3311C4C230C772394
:10520000B03CE6F59C3B10235013908C2FA2589590
:105210000206ED80A61C58A6B9A0FE4FE61B5C5006
:10522000DC985C5B0E4EDC605090461F1A171ACE5D
:105230001A7B19A4BC9CA27CA863F9104E9CA23CCA
:105240000B4E9CA20E1CD0BC305A1CD0BC70B03D82
:10525000ACAE7E4484C4FE1F88C83EAE7EFE1F48AE
:10526000C83EE089284C2BA66DAC7B58A6D5C00E55
:105270003C3370D8F0D826AAD3B0E01CA28103A298
:1052800013C88CAB998C949FB9A00EFEDFE6AB4E91
:10529000DC909050A646171AC12E605C021B76CE99
:1052A000CEFA027C9C02A388465E7C464BFCA64656
:1052B0002BFCA64627069D2E1C026DA001A484444B
:1052C000CC0D2F6E0C770C67089DCCC8CCB1234950
:1052D0004C2922B85CE22F9CE2ADBE9C154E26BC48
:1052E00030D61BBEBE0630501C0A4F30304A7C1CE4
:1052F000D0D05BAA1C109016E217625C7C66EBD8DB
:1053000084D806101CAA027390BC1C10B61B901304
:10531000D09090612E0AFC5A7A7C5CE227D05C1314
:105320009CB6AF10B67FB67FE6E6B62B101C903B5E
:105330005056DB1B9013D0FB1CD0D0E61630A006D5
:10534000CFC6E676541B5C23FC9CD08C1F50139078
:10535000EAAA1C224BD01CAAE0E65CD0A362A6BE3F
:10536000B33A46F12E84A04E30493606F3600DA4C0
:10537000E6CBEEAE0EBCFA4EDC901AEE1A7E3F1A69
:10538000FAFA1AFAB31ABA30FFDC90FE061C707EE5
:105390009E387C361FBA573CBED3A62A77A6067B1A
:1053A0007E9EBEBCB6CA6A3736275C194E7601A40B
:1053B000A6AD9C059C0679A431A48C092B0C470C46
:1053C00037B85E5AA84EA6E81936981BB07C869C62
:1053D00006301070603008626F787C0C2B06300548
:1053E000463C301B3362783C62F3661C56E66036FE
:1053F000E05CD0D0F92E00000000300A0660C9261B
:10540000150E7EFE8DD77C0EE12A39CC663006065D
:10541000A5A84E705B3009512C067CA5A8301070F1
:105420004E2868A893F980CDA8619C0821BC934EB2
:105430007019A410A8489502F980CDA80821BC0EC7
:10544000B09926F910A079A4FA5C5050D010D05031
:1054500090909050237AFA7ADC133A62F354BB6945
:10546000483A38BA28BA4E66FD3963F910A079A4D3
:10547000ABF980F6332627DAFAE7BA79A4BAF0B0A6
:105480006B45BE8889284CF1CB095699AC99AC99EB
:10549000ACE3F910C1CCBBF91011A0EE3A467BF990
:1054A000100C4319BC5821BC98F06DA4F86D02E5AE
:1054B000ACE35EE0C84801504C378C3301A0CB8C84
:1054C000605E054479404CB3E14CE140CC6735382F
:1054D000AE58B01E98BE1EAEE0A18879400D3C6D5E
:1054E00040CC1F353AE14C4B01A0F5407940B0016A
:1054F000A01138993C6D40B54A01508C600E5CA2F9
:105500004A2F4E7A365B0EFD401E7940B05E01A0F8
:10551000F940553CB548513201508C60CD38794046
:1055200031887940553CB05E0540B548CB19ACF1A7
:105530000201A4E677B1A80DA4440C9F0C9779CC86
:1055400084B3CC2B81008C2B6E65CC6E65220484D9
:10555000C1CCE637EED704BD02F637B19601A40CF4
:10556000570CCF0884E6B123C51EF59C844B45BC7F
:10557000E04554461C1066FB0C15A1950235528877
:105580007DACD180280E4C23C1AC1BC9ACE9CC2D1D
:105590004059A438CD384C23BDAC1BC5ACE9CC3543
:1055A0004059A44C1F48F30EB08538E9CCB9AC354E
:1055B000400E62E9CCCDAC2D40D59CF1027DAC31E2
:1055C000ACC1ACAEFA271C154E7D3CEDA831ACC980
:1055D000ACAE7D3C6D027DAC44CDAC2EFAAE8540C8
:1055E00079404C272D401BC540B14CDD40C14CA13A
:1055F0004C4C27284823EDA838DB7DACD9A03D0EC4
:105600007DAC090C837DACC9ACEEC1ACF5A8EE2B2A
:105610000CC748B38CDF4806B07DA01C625BEADC97
:10562000E38C1F44A30CAF8BA214FFD4274C177E2E
:10563000D4D48EAAEE3CDCCABCAEEE5C1EA05AAF3F
:105640000EAE6E738C1B0CC7FAA1028928CCD1CB8D
:10565000BE44F0B34267A6FAE326935CEA8EB0A09C
:105660009CC54086061CD62B8A838A06AEFCAE26D5
:105670001C5E2FA6EE8ADBA66E6544546D029B9CD1
:10568000A2A2A2D384488CD789A0442E5C22029C7B
:10569000D84670F8AAA6E8A6AAD86A085A0F046ADB
:1056A000F3FA13EEDCD0EE3EB30CA72E1B0E6B19F3
:1056B0004A0546F54A0EA14884B08D38514EFD404A
:1056C000230EBEC74D40CB4E5C665093DD408BDD54
:1056D000805D28CC7DC32BD18066662E7A58463EED
:1056E0005ED8065E139E0ED8DCDC8E132E62F35459
:1056F000CB98AE58FE1B66CEAE5C4AD7EEAE5C0EC3
:10570000E66B3A5BC62622DE6EFA604E1EE0C6C32A
:105710004D40A06E4B423766EAE30E11A0EEB08D0D
:1057200038A500C30EA500853811A093881D448CB0
:105730004B98D44A538928CC9DC72EFAAE4ED84EEA
:105740005C50EEAED8AEBBFABB693CB36140A34D32
:105750004063DD805D28CCA1C32E7A58463EFAA175
:105760003ED8465E139ED85EAE6E2E2BD8EE66D81F
:105770005C4E13228EF32EEED4D4D3AE98093E5D48
:10578000384502F5484E58A148EE9BD180F5403887
:1057900066660043C1405BA140432980232EFAAED8
:1057A0007E239C154E1E3ECEEE113E6EEEEE0EEEAC
:1057B0005A0EE62BAEBA0EEEEE4E9C4217AE8E4E51
:1057C0006EDC50CE4B22CEF34EEE94F7D4CAC3C853
:1057D00048A5A07D1AC848C8A5A0B916A5A07516E9
:1057E000A5A025168809A642231013503C1EF8FCDC
:1057F000D88404D83C601EE895026544F08CA0195A
:10580000A45C84903B2E7A05406544F0FB5C500517
:10581000403B0E2E7AE32D404E7078A83868CEBEFD
:105820001E28F8BA9CEAEAEABAE8AA8A8A8AEBF160
:10583000404E70EED8F81A9ABABABA1CEAE6E838BE
:10584000EE7828B868BA463CFED8EE5CE030049C9E
:10585000737030051C4BA1881B794030069C703852
:10586000EED8F8D4CE14EBFEAED80BC1AC1D38790F
:105870004031ACBDACDBC9ACAEC1AC21387940CD58
:10588000ACAEB9AC63C9AC1D387940CDACAEC5ACDB
:105890008538DD404B4D40EB4E231E4EBE5C50E341
:1058A000DD805D28CC29C393DD805D28CC4DC34BC2
:1058B000BE5761404B0E78AEBE2E7A58463E5ED83B
:1058C0001CD4763654E3EEEE6BD86EEE4B2687D8BA
:1058D0006E26DFAED80E23D8AE2BD8AED86E9E5E25
:1058E0005B8E1E263BD8FCD86EA66E264B66CEBEBF
:1058F0001ED4D4C34EAE98EE2E767676767600E140
:105900003A2EFAAEA0DCCED86ECEF66026E63B6626
:10591000EE1ED44ECF66E0A643A13EFEEFF6DF0EAC
:105920008E1CEE8A5C4A8F66061B36E04E22CE3E07
:10593000EEC21BAA260EC223EE2EFBDE338A6E2693
:105940002EFB6A626B7E5BEE865A5E2A4EBAE04D93
:10595000408D3CFA174EA05CF62B86F61F86E0F6CB
:105960001F4E334A6A5688D4D4E0BE6E8E588E4E8F
:1059700027980EE026CB5C626EC13E2EFAAE840400
:105980005E13081E1A6ECEE673CE5E7FDCD4947969
:105990004726DBDD48C3A1485C336E66AE333A8EE2
:1059A000F32EEE66539CE22B62E24F225C43AEFA8A
:1059B000AEE26B4E5C6A0E1C500C13A66E0E4C3B96
:1059C00079408540A1888C1BBE1E653E228EF32E39
:1059D0005447EE66D4EE6546EE4C2B4948AE6EDC7D
:1059E000909CFAABDCE22B628E58E3268E7EA346B7
:1059F0003C626E0E0C0D3D3B6E5A5E0E0CC1454C6A
:105A00007941794013AE7EF32E7E98D3588EEEEE18
:105A1000EE0E6ECEEE2798AEE066CB8ED826B13E67
:105A20000EEE5C90D01090501050105090505010CE
:105A30000B4E54977A103AD4DF5437147F94BF54E6
:105A4000E79CD05C6B9050D05010D050101050900C
:105A50005CEEE0D0501050D050101010D0D09C937D
:105A60001CD0D0101050D03068DC3B5CD0D0D010AF
:105A700010D0505CEB5CD0D030311CB330339C93F1
:105A80002EFAAE794084D1805EBB06BAF633A13ED1
:105A9000E6EB66EE5ADFE64FBE1EFEFE1EFE1388E4
:105AA00059A45EB54845022EFAAE48DA7FDD40FAC9
:105AB000F398FEDF2E653E2EFAAE44043E7E871E2E
:105AC000DA6BA606E67B461BA6080E5E5A5C8A6267
:105AD000228E588B5CCE62AE4E314E422766EEE38C
:105AE000D8C13C8B7940AB44043EAE0E26E6B35E93
:105AF00057AEC5445C4EA60E6E3B08CB54F7D43E61
:105B000026DB7B8E7EF3982EBE3B3E6EEED4949BBE
:105B1000AE8EEAEAEAAE9CD086C6DB5C8EEEDD484D
:105B2000894CFAE3D4BB2E9C822E8E9D480C376E96
:105B30008E6E2E6E1C894CFA3B8EDBEED38E235E6E
:105B4000EF665E0CF519FD384CA0DD40953898FEE7
:105B50001546A6EEDB8E49486E5C232E62F3422684
:105B6000DCE05E47993ECDAC5846FA31368D3E8535
:105B700040E36140CB66665C4227FAA6E3AEE08470
:105B8000A00404C4A01BD46694EB606EE6A2561772
:105B9000B6A61C9090901090BCAE1C55544C290396
:105BA0008C2F0C603D4C4E70606E28F83051A6E88A
:105BB00060001C4610662FC8CCE7934EA8DC90907E
:105BC0001C1010D0109068959EC8CCF73004C8CC3B
:105BD00066EBE09CA20242300842DCCC2799A82365
:105BE00099A8B6B6B6B699067940658C29381E993B
:105BF0003CDD428BE5D3C6F50000EE4BF643A63004
:105C00000786061388D9A2F6FFB9A00EB0CEFE2FE4
:105C10004E8F85464E375C4A2236E0E65B66E643A9
:105C20004EE0E62366E687F5CC0EB0FD407940797C
:105C30004029384E5090268D3879404E5C26505081
:105C40000540D15C1050213C4E26D010D0101005DC
:105C5000406D40D15C50D0213C4E269050D05050E9
:105C6000554061404E5CD08D3861404EBED84E10DC
:105C70001010213C4E106605416D40E14C4E66D837
:105C80004E50501050D01050D0D09010D00D4061D8
:105C900040F1CC0D40A18861404EBE664D4185402B
:105CA00001484938614011447940F5CC2EFA0E790B
:105CB00040DA5BB00540E14CA18885409B614065BE
:105CC0003E143F8CD532600CD7DC501C6233542715
:105CD000DC7ED34C3B7E37A2D4442BBE025437B07B
:105CE000E13A069C4A3704F80AA1025C4A279C0262
:105CF000138A8D3AFE2F1D444EA0A13E15A0D180DF
:105D0000E95059A4E9503DACB01C427FF940FE5F18
:105D1000680EB0288C4FF940FE2B7828B06859A443
:105D20005CEE1F502B4E50280E78FD407940785580
:105D3000A46E9B2E7A7940680EB8FD40788C853C25
:105D40004938F637434D40653C45025CC44813442E
:105D5000846095584E70E0DCD0AE281E5F7E530CF8
:105D60003B9CE21FD013D05EA83C0E364F85BCD6BC
:105D70001B5C903C4EB83C365F85BCD61B9C107CAF
:105D8000EEEE4EB83C364F85BCD61B1C103C4EB8D0
:105D90007C364F85BCD61B9C10FC4EB8BC36578554
:105DA000BCD61390FCEEEE4EAE91580EB87C365F2A
:105DB00085BCD61B5C90BCEEEE4EB8BC364F85BCA5
:105DC000D61B5C90BC4EB83C365F85BCD61B9C1085
:105DD0003CEEEE4EB87C365F85BCD61B5C107CEE8C
:105DE000EE4EB8FC367F1CE22371BC1B85BCD61B73
:105DF0009C10FC4EAE7D588C234CFD5BF8FE434E50
:105E00003008A8300C3B4E300CA8300868A0381E73
:105E10007E077E9F7EC77E677ED35C22AFB87CEE16
:105E2000EE0E7B787C4EB8BCEEEE4E7C1B787C4E42
:105E30006E1D5A4DDC0EFC9C02788C234C174EA232
:105E400097A20FA25FA27FA2F7A25FA27FA2F7A2F2
:105E5000477B7C4EB87CEEEE4E6EB87CEEEE4EB8D4
:105E6000BC4EC37C4EB8BCEEEE4E6EB83C4E637C6E
:105E7000EEEE4E6EB87C4EB8BC4E9CB0FE23109C2D
:105E8000427870686E89588C1B4C7FF85A460C1B00
:105E90001C50FEFE3B1C10FE1B1C105EDC8C1350C5
:105EA0008558F8FC5A46FE235C505E1CCC1B223BF6
:105EB000A09423E01C50E07158380E8E5C505C6258
:105EC0004F78BCD88404D8BC68E0208C3F19A45C0F
:105ED000E21330A059A60E7870682B0EB870A88C0B
:105EE0002BCCA048E04C60C8CC6088494EA01C1068
:105EF0009C50201378EE68A8863D4C4E5C906EFF57
:105F0000CCEB30DA065ABC3006203C56668F6E6603
:105F10003028060F4E6E1C50500E55549502664E9A
:105F2000A02660A6E33C315E15A0B028C444415CC5
:105F3000D50CAEF0986EBFA01C100626E630187C7B
:105F4000BA5CCC2B62622222304613263A7AD7867C
:105F5000465F48415CB0CE4E3A30F3A6CC231C904D
:105F6000106E5FD50C0E986E2FCC2FC80B4E834E43
:105F70007038704E6E68A8CCA08481024E2626CC64
:105F80001B26263C134E5CF0154EA0D50CF0F0D825
:105F9000D8D8D8D8D8EE6ED50CCE4E5758844E30BF
:105FA00007CC2388301A70EE384EAE8C274C7F2EEB
:105FB000AED8F04E38D8F06E3019667784302A4C5F
:105FC00017860698065830187B30E0CC1B30C06628
:105FD000833010662730E0066EEE6656538E008BD7
:105FE0006EE0584E7078A84E7038689828E04EBE23
:105FF0002626D84EDC5050905CE03D8540EBBBBA85
:10600000974F3F4361407180A18871806D427D8CC4
:1060100051A91A27C78DAE0E58CE6B79894DB58818
:106020004D40B005405D4021BC05426F66743DACFB
:10603000B0E580AE236DA4B87EFE271C154E3EE071
:10604000CC24525B906140953A918863B58838BE04
:106050002878BE6863B5884D40B08D38F1886140BE
:1060600021BCBE8D391DB8F0E9808D38A18821BCD6
:106070008D38614058C98898E078BE681E61401E1E
:106080000D40FAA13E858AFD803BFD80BD8875806C
:1060900019BC318C6DA4F8CD8C3180C988493C5D28
:1060A00040D54E9188B0FE1348813CB05E05403526
:1060B00038993C70FAA0DDACE14C1E4CA05EF0BEFD
:1060C000E0D180E1AC70FA2F21BCFA2B01BCFAAF11
:1060D000198C1E21BCFA2BD188886B7940198CE170
:1060E000AC703988DD40A188B0318CF18884C1481A
:1060F0008588C9884938B1A861882D80619C704D18
:10610000402D80EBD58884BD88858875808C43D9E7
:106110008461883B9188D98459882D805D402938D5
:106120002B21BCFA2FED3859028DD899487940D3EC
:106130004D40441144A1886142D588984BD5889937
:106140004879408580798E884D8C1B91888D84C9D3
:10615000882938C9880580F1887D808C4BF0BE374E
:10616000E988FA1BFEC3BEF0EB4D8CF588834D8C9D
:1061700065845B884D8C1B91888D842D8070854053
:106180002938CB4D8C1B91888D8429385D40058042
:10619000739188C988418CC9883180FA276D1C9B0E
:1061A00021BC5E5846213C4E108D38B5485C4E10DF
:1061B000853C0E21BC1EAE5D404E9005402D806D8D
:1061C00040F1CC7140DDACC988318859A478FA1F00
:1061D000B01E3538F0E09188813C704EE021BC70F3
:1061E000ED308C2B318C79407140AE0EDA70048C1E
:1061F000130859880C17847D40A606DA6544845438
:1062000027D4472E71807940993E1EE04484C4E033
:1062100048888849886EEE711A0C4321BC5819BC15
:1062200098F06DA4B0E8E09188619CAE70E08819A8
:106230008C4EAE900EB05EFD40FE33298001487B4F
:106240004D408540A188794049383980B5488588D6
:10625000A188198C8C1F4888398870C988F1886199
:1062600084584E70F83CA6BCE83004A34E70F87C0D
:10627000A63CE83005534E70F87CA6BCE8300670AA
:1062800038BE5CEAF0E048884988884D40DA8B5E89
:10629000231E88C8E14CFA170EFE1348C8ED16619C
:1062A000400611A04C4F4E668C2366501350EEFAF8
:1062B000653FA0E0C891881E7940794085403180D3
:1062C000993C794085401E79406D40E14CA188851C
:1062D00040418C71801DB8993C4D401E0D40F188A5
:1062E0008540DA213DE140F188E140DD4098FE1B28
:1062F000C988DD407940658CA1883538B94C0D409E
:10630000B5480E21BCFA1FB0BE1EAECC13BEFA17A4
:106310005EF048C848884484318C6140D54C79404F
:106320004EAE698DFE676140DDAC8540213CC514F1
:106330000B6140A188CC2388C413C8F1CCB94CC5EB
:1063400014DD4098FE53F1CC8C3311A0EE0D406566
:106350003CF0E04E5C900542D8EED8B07EFE439C07
:10636000C23F59A47EFE252298666666064E309E80
:106370001C90BC70A65A1C90BC305A1C90BC70A0DB
:1063800021BC58318CB0CD8C79428140E321BC587E
:10639000B0F0918898BE704B65445821BC98F0B01D
:1063A0006D02FCFEDEFC06512CE6A675AC31DC6607
:1063B00081CCFA3C0681CCBC1A60DECE9C4A6A3A9B
:1063C000CC1BD0D0C49CAAE217D09CD0E217D0DC62
:1063D000D00EE0B05E5CD4A6F3E0CC1FC8E0C4E011
:1063E0006DA45CB87EFE2F0E7C9C023EE00E2E7AE1
:1063F000E0A7DBD3E8D07100000002A628D1808995
:10640000900C1F0C930DA4BCE6852BBCAECC374C76
:10641000339C154E8CE7CC2355A8238C61A844846B
:106420004E7038066DA0860DA40C570C470E5E5AB0
:10643000A84EE88BF59C0E1CA2B86190AEC6E8B8D9
:106440001CAAAEA8A0844D90CC01B27CC6BCE83D8D
:10645000AC91A44EF0688DACAE5891A49828F94048
:106460004E6828DAE59A3538380540700666667851
:10647000F0EE0D107D88EE70E9907C2370E990A617
:106480006DA4AEE89DA4840C270C2F084CB12230DB
:10649000BD02CEBEEECEBEEECEBEEEE044840DA476
:1064A0000E1C0A3003E6F86190E6A0F6DF06261F10
:1064B00088B348A36601A4BEBAB06544848DAC1904
:1064C000AC19AC700DA4EECE61901CCAA8A9A43C76
:1064D000E091A4B0FA274626765C5A5E50EE4E1C38
:1064E00098163C422666E21B4213A6566F58860653
:1064F00046B6504626561B26986E46E09DA44EF0A2
:106500005D90B0A8AEA85C4E90E8A9A45E46F0915C
:10651000A44E68E8380EB8FD4068380E78F540782B
:106520008D383D40844E22E80EF8F540FEFD97F888
:10653000853C718028F80EFD40F80540388D38F80C
:10654000853C4E669041387038ED40B08D38700E05
:1065500038FD40F0ED4028066648CD925D90AEA82B
:1065600038F02806669B0E46E8E0B0A0A6A6A1B3C8
:10657000A645B7A60997A62F5D90B8FD40A8F80ECE
:10658000F87D3C718085404EBE504138794091A4E1
:10659000B88D38F80540E8380E78F01138B0FED8DC
:1065A000A9A4FED80D407940A9A4A6F07E91A4CE5E
:1065B000684E900EF8FD40B596F81D3868F80EF854
:1065C0007D3CF0B80E787D3CB8D940B005403538F8
:1065D000B80540A84D409DA47091A4F8853CB8D959
:1065E00040B0554091A4B80EF0FD4078853C614024
:1065F0006184554091A4B870F8FA23DA50260EE869
:106600008538854085A4B0AE7D3CB00540A8619C2E
:106610002E7A553C6D40709E91A4CE68A9A4A60622
:10662000F0B0D94058388DA4AEE89828B80EB0F52F
:106630004068B0A888084EA8F84AFC0E4E1CD0E866
:10664000901C029C48021BAE44F08C1F041384B8BB
:106650000E4E5C1085384ED00540A8380EF87038C4
:10666000F94091A4780540E8B80EE0DCA01CF25295
:106670005E1B6692F85EF940FE238408F80EB09C1B
:1066800002D3AE70AE38BEAE227038FD4091A4B8D1
:106690008D38F8853C4E90D940FE1B8808380EF89E
:1066A00070AEF091A4F80EB87D3C38054028F80E85
:1066B0000CCBB0AE9C22E802419AF80E4C3738AEB3
:1066C00070AEF0A9A43E4D967EEF3885A47819AC43
:1066D000F54091A4B870389D88980EB01138704D6F
:1066E000401E91A4B88D38B0FA435A5E5066D41457
:1066F000EB35408DACB001401D9CEE559304041564
:10670000322E44601C0DA4EA0EF861901CE21F04B6
:106710001322E89DA4AE1CEAA8F8E005A8452409C8
:106720009CB8F61F1CD0061CD0B656F6A678FD9C69
:10673000B806FD9CEE7C5CD0231C6124E61F7ECE57
:10674000BC76FABCFAE08C2788A922849502F85C12
:10675000A2E8D38C27B07EFEE1025E7E0E45543D5A
:106760004CE5368CA70C75CE21BCF05845BC455481
:1067700098706B0C1F0CA030107038A0266028F8A1
:10678000E633DDA4229D9D301070B806F866BF3850
:1067900029A446E33D9CE6A03D9CE6B3DDA422018E
:1067A000A7301070F81CE65316D0164BB636DCF046
:1067B000E030FFDB661C50BB0DA45B79A4F1A4E6BE
:1067C000A7B806F8A6E89DA47376F6371CD02A135E
:1067D00046F3EE0C8311BCAE09BCAEF001BCAEF0CA
:1067E00021BCAEF059A40E7828B868EEE0EEB30EE6
:1067F0007D88AEE00000000000000E5C62E04ED834
:1068000061A0EECEE0FC5C34CC7460A0494CCC605E
:1068100060005C4ED01050D050105090D0D050D06E
:10682000505CE0F8448460FEFE2BFE174888A05CB4
:10683000B0F9820C5F0C4FC1CCA18C4554E14CEEF9
:106840004E70DCD010901010D01010684E5C1010FC
:10685000D010D01090A8EE30E00C1720608C60F9BA
:106860001004881A1EBA4EE01D4498D44AFA1BE65A
:10687000FEE0AED8601E1A3A79A4FE8B4E4651A2B5
:106880009CB6FC1A7C1EBE66660676CB2213BA3610
:1068900013BA7C2213BA3613BA7C2213BA3613BA4F
:1068A0007C2213BAA666067038261363E62B5A7C40
:1068B0000E66072213BA3CBEDB4EA6A65606E606B7
:1068C000E606BC1A3C0681CC605EFADABC0E79A4FE
:1068D00031A45CAAE060660DA4E6C12E5A5C50FAB1
:1068E0007658F8761CEA1F30FF1A0698DC901C6A6E
:1068F0001F883CBE9EA6065670381BBE3CB6EB6693
:106900006A833CBEE3661A8C334C874884D3A61650
:10691000DB3ED31A3A9F565F7E9E7EBEBCF66684EF
:106920004430107038DCD08B56CB7E6B3A4B569B84
:1069300066661CD01653A06660283017AB301693DD
:10694000301A1C73469BAEAEAEC65E6B30151B0E86
:106950004E7038E00E3010D33014BB8DAC0E3020AA
:106960008B30307330035B30214330222B0E3023C9
:106970000B9C06567038B6133CB6F3E0FAA00E8EA8
:106980002626065C4647D4941BCEE066D34EDA8CAE
:1069900093DCD423B51C2BDCB51CD4D4B51C0ECE93
:1069A000E13A0EAD1CDCD417DCAD1CEE4EEE93EAE2
:1069B000EA8E8E7388AEDCD4BBCE667038AEFC1C1B
:1069C0000ADC7CAEF073B1A80DA45AFCC658F8E6F8
:1069D000A922769C1BDCDC76EB5670EE3822B7DC05
:1069E000AEEAEA8E8E986E9C8CA35C93A6AE0E7077
:1069F000383C8C133CAE6A2670AEF0A6986677AE33
:106A000070EEBA5A3B8C2BBA5A174EF00DA43D9C2F
:106A10008C3D9D059C91CC8495025C44E616864B8A
:106A200089A888E05C0644448484C4C4E00C600502
:106A3000A849A47C56063016C6A6D349A46044844F
:106A40007C061C301B6AA089908C2F4C3746333053
:106A50001C1B300A064E3008581A7A8E2B0EFC1674
:106A6000AE583C75ACBA3CE61C4A23CA1F06264207
:106A700033C223DC154E4EC6BC1A8EE6EEEE98BA33
:106A800058CE0E3A462635CC7CC92CC65ABCA60632
:106A9000BC1A6E983CFE78C92C0EB8C92C26A606E6
:106AA0009F6E78EE4EA606561C3B6E4A7CDCDC6E72
:106AB0007ECB6E78C92CE6AE68B86EEE983C1EDCD4
:106AC000901ECF7EFC5C7E67FCDC7E47EE78EE9C01
:106AD0003C7E93EAD4D4D4D4EACEF0AEE63CA63CD5
:106AE000A6ADAC56602E1C336A70EEF0EE6AD7E0AD
:106AF00019A4E2674B65440E4CBFB019AC0D10AE43
:106B0000A15C5C0CA021BCD801BCD8F009BCD8F0B9
:106B100011BCD8F059A619A45CE2D310BB0D100B20
:106B20005821BC619CEE98A80C3B11BCEEF04E7055
:106B3000AEE0B00C730E21BC5801BCD8F021BCD81B
:106B4000F0AE3DACF05BCDAC43AE4E70381BB07CCC
:106B50009C62A03CA28DA8412C06983C512CC6E614
:106B60007CC92CA666E6F1BE5A3C66C646BC1AF63F
:106B70009F86465BEE6670EE38AE6670AEF0BAABDE
:106B800066C6E066A68646005BEE2670EE38AE2648
:106B900070AEF0BAAB66C626E039CCEE7026EE38A1
:106BA000F980DC94BB5CB02BD4D4D4D4D460301046
:106BB00070787C561B26DC54EB70388B4D40DD40E2
:106BC0003856703860F62BA05676E056A0E0984311
:106BD000B00E4D2CEEAE7C0E3010709CB8603C6256
:106BE0007C62477C622F783C62BB3C5A7CC60E1CA0
:106BF000E0EE5CEA23CE5066EEE0C61CD0BCE89125
:106C0000A44EA8E8B0283DAC4EEEA74E6F91A4BDAF
:106C1000DC9CD08668280609925C621BA2A291A423
:106C2000AE9BEE9785A43819AC43B085A419ACB5DA
:106C3000A4F084F99A70D1A4EEA9B60EB05EFED588
:106C4000B71EF940FE17EEDDB2C1A4EE63A9A45C45
:106C500002D05C620213A2E8D1A4A878283868B0F8
:106C6000E8F8B9DC3A853879404DB8EE6B55449177
:106C7000D8BDDC2626D940FE3FBDDC262691D89122
:106C8000A40E78F54079402D80B5A455406140D8D8
:106C90005EFECB4D404E3E6E8D387DB8EE5F61405E
:106CA000B5A405407DB8EEB338C1B64D40BDDC3A61
:106CB00043C1A4EE2FB0A89DB2A9A45CE225B662A0
:106CC000E829B87940B0CDA4F9404D40213C794045
:106CD0004DB8794039B8553CBE1EE140A18891A419
:106CE0000E38F540553C3ECE43E14CBE1E1DB81B50
:106CF000854075B4EE57854075B4EE2738282B389B
:106D00004EEE27D1A485A48DACB5A4F01D9CEE2F2A
:106D10001C0C154E8481023538B5A4054065B82891
:106D20000E784EE0B0E84EA891A42806480992F8E3
:106D3000A8786DB82884B0E838688DA4F940794007
:106D4000C1A40EF87D3CBDDC3AD940553C0EB5A43B
:106D5000FD407DB8EE2F39B8B5A45CFA37BEB62633
:106D6000228B5E37FE373A5BBBFEE762FA1B2213CB
:106D7000667A0065B8284EEEC1B2B870388DA44E60
:106D8000EE27B08C5BAE0E0666C9B6EEA9B270CD2A
:106D9000A45EFED5B7F8AE7D3C8540794091A40E47
:106DA00038F9402938794029B85544B9DCF9406DA3
:106DB000B8A8EDB4F940FE1BC1A45EA8EDB4FD4037
:106DC0007940C1A4B9DCFD40553C7940F1B486D985
:106DD00041FEEB4D40B0BE8D3983C1A4EDB486F9C0
:106DE00041FE6BC1A40EB0213865B8A888F1B6B0D9
:106DF000262626BEAF0EBDDC666666E07910A00DC5
:106E0000428540DB91A4381B91A40E782BC1A40EBF
:106E1000F8F94265448DA4AEE065B80E28784EE0DE
:106E2000E6461CA2E6E6E6C6029CE24B300A9C025D
:106E30001F881376E6E0301246865CC4C61DAC0E91
:106E4000B0E0481C02300AB68CB70A23F6134A3069
:106E500002C62749A47C56467CC92C0675CEDB3079
:106E600012A69C2222A7998C9437B9A0D1B80B1AEC
:106E7000AE5859A44C6DA4FA23F617EEB04C17780F
:106E8000F6DFFACBD1B89A9A981A58CE8ED1B89824
:106E90001A58AE5ABCFA51AC3A1F260F986E2637D4
:106EA000363A1736586ECE35CC9816860CC70CB7C6
:106EB0003C5C4A6ADCD09CD0E217D00E1CE217EA98
:106EC000664554E14C9C09BA6DA478A076B66FB6BD
:106ED0009F0C1F0C13C479B884CD3C01A01EFD404B
:106EE000F06DA679B8B3F6134E066606E5AB7EFEE6
:106EF00005825E66601ADC0AF62B9A02FC53E6896C
:106F0000BB7CE606E6E64646FC46E084B07EFEA193
:106F10008E3EEE8C6084049C981CE2330862E2137F
:106F20008860069CA24670300A061706A0CE660C42
:106F30003756B7301006D326061F6606658CF61343
:106F4000DC6DBC281E56074B66866646874E3E1390
:106F5000B0280861BC2361BC288CF7F623A0867694
:106F6000A69CEAEAEA73FE1FFA4B8E26F32B7EA656
:106F700046EF608438DE06E0E676A63030C6FB4693
:106F8000C6C6FB46C65C13A2A6977EA066D4606206
:106F9000BBBB66658C0E0A5A137E0ABEBAFE930C02
:106FA000BB26F64B76F62FB00E1E5B36A6CEA60697
:106FB0001E1A60AA06A0E026D49BDC435C331C2387
:106FC0009C139C3010707830097C366066DC54EB82
:106FD000F617A0565DA65A9C90102B5A5CD0D0FC98
:106FE00030F65A56E0F59C0E1CA2B8619066AEE8E9
:106FF000B81CAAAEA8BD02000000D4CCE23A2EC54F
:10700000D4AEEE8E4C2B8CFDC3AE44841B4C3B8C1B
:1070100001C3AE4813444488BB4C2B8C69C3AE48B3
:1070200084734C438C99D7447CA9C6EEA13E485842
:10703000A9A45CA2E8E5A0F80E986E19DC6EFDDC50
:10704000AE55ACFDDCD5C06A173CC9DCAE281DAC22
:10705000AE4C5F8C334C13AEBE00FD40438C278595
:10706000381B7D3C3D4081C47CF3C1CC45027C5142
:107070002C7C0A3C56CA7CAAE0446E71ACEE71AC22
:107080006E5C85D4EDDC55A47C9C6251AD59A4D1D5
:10709000C07C0E492CAEAA3CF9DC512CAEAA3C6A4D
:1070A000C1C315DC0E1DACAE3C581DACD83C5670AF
:1070B000984CF5192D40C9DC1C2A3C2A3C26034C6F
:1070C0007B8C6B8483E6E63C56FEA00DC8134C8D8A
:1070D000D68CEB447C58BA5DD4A6D8629BD875ACEC
:1070E000FCC68C2F7CA6FCA6D875AC98FCA6587C58
:1070F00079D44C5FFDDC75AC986AAF3C79D4EDDC9B
:10710000D819DC063CE6B9A8412CC9DC7C1CAAFCD9
:1071100055A44D2CAA492CAEFCAAFC06668C170A75
:107120006AC1C37CEACAFCEA6A07FCEE7E79401CAD
:107130007EEEAA41DC09AC4C27F1CC134E35404D14
:10714000407EEE8DC47C2A7C033C6A0A3CEDC0067E
:10715000667C8C130A7C0A7C6A3B467038601C2A69
:10716000E08445D475AC3C85D4EDDC0E51ACC1CC8B
:1071700029DCCC2701D0688C9739CCB1D0C1CC4C5C
:1071800025C755A4488401C288CBBDDCCD8CA1881D
:10719000C9DC163CB6765FFC68CDDCC9DC3CDE3C65
:1071A0005EA04D40D8FEF1CD781DAC8D381C107618
:1071B00027B60AAA36761F760AA188786079DC3C61
:1071C000AB593C0E65026DA4BDDCF0688102300E47
:1071D00058A0B9A8300906986666B78B45D4CDCCBF
:1071E000C5CC0DC851ACE62DC0CDCCC9DC063CC623
:1071F00091AC51ACEEEEEEDAC6E6C6BCC9DCBA1A0A
:107200009C0A26FB70EE38AE70D83845DCAEF0EE46
:1072100070D8AEF0D86626BA63661A0A3C4666464F
:10722000BCC67C661F3C8BB045D40DC88102447C33
:107230005871C8CBC48845D40DC8D5CC7371C8412A
:107240002C0A3CAA3CEE51ACEA5B3CEEAA3CEA3C80
:107250002A0A7C6AE315DC85DCCC973836F031DC11
:10726000781C0A3CCA3C4A7CAA0AFC0A2FCA7C2A1F
:10727000BB3CEACA7C0A7C4A7C6A1F2AEB7CAA686F
:107280000EB8AE85DC3836AEF0AECC9BC9DC1C0B3C
:1072900051ACE63C29CC98D5C06A603C0E1DAC4C84
:1072A00045DCF060AE2A7C937D884CC315A059ACB8
:1072B000467CA6BCEE704E7028EEEB701DAC5E05F1
:1072C0004060B0267AB3707940614009B8604D40A3
:1072D000D8FEC989DD4078663F680EB0BA2E3359B2
:1072E0003C6D02F59CB05ED37D884CC315A08DD853
:1072F000B0D1C06A7715DC1DAC0E85DCC9DC1C2A58
:107300007C934D40A0993CD3C9DC5E5A3C3616FCB8
:1073100016A358CDDCFE983C16FCDCB65623D4AE42
:10732000DBC279DC43C9DCBEBA68E0881384C45987
:10733000AC3CE68C2DC1EE3CA63CC619DC7CCC2BCB
:10734000E68C2DC006B9AA3C660613A6BC668E065E
:1073500013267AF3412C46E02679A429A42301A41C
:10736000E60DA45E5AA84EE6E8E0B80E60F861901B
:107370001CE21322E89DA45C8A8A8AAEA8AEE0B122
:1073800020F8E637300CE8E6E6C8CC2366E3E049AF
:107390004CB14E301070F86006E6A01CD076175C39
:1073A000E5A4FC16FC366B54277CB6E0A6065666B0
:1073B0007038C3763C56E0B0BE0E4E5CD0FD40FE49
:1073C0008541B9A0FE134EE049A4607C0616867C78
:1073D000A61CCA30060AA01C154E4EDC90A01AEE60
:1073E0007ABA1A7E60FAFAFAFAAB301070B87C5AA0
:1073F000463C3EE08CA0BEBEBEE0C9DC42F5DC36B9
:10740000605C42FC1C5050507CB9DC367F11D8C9FE
:10741000DCFC5AAB0617A67683A67302A242E35C95
:1074200090681C509C55DC41DC02170241DC62353F
:10743000D8B815D801D8ADDC36439C55DC55DC11E5
:10744000D82DDC78B9DC36B711D8DC50DDDCA0FDF6
:1074500040FE8BF8FC1DAC2DDC7851DC433C16FC67
:10746000B63C681E7C7E4B781C02A241DC21D87899
:1074700061D831DCA0FA6778767647FCB9DC1C224B
:1074800046A8B8C9DC58B6167EF63B7E3FFE1FB64E
:107490001BBC56AE09D898D9DC360DD311D8DDDC2B
:1074A000A07D3CADDCA3C9DCF6A05C42B9DC36E7CC
:1074B00039DC68EDDC36B7683DDC6251DC2235D85A
:1074C00035D861400D4045DC01D84B163CB67C39BF
:1074D000DC6841D8013CBDDC62E2AB683C16767CDE
:1074E000B63C163C2DD8B861D8BEC1D5A9DC535CDA
:1074F00062E2EF9C505C50685C02EE9C02533C16CA
:107500007CB6FC25D84E4351DC2225D835D86140C5
:1075100011B8A9DCB9DC7636FFF5DC36CB163CB603
:10752000BC68C9DC62E2A0E5D862D368028E8E1C1A
:10753000A20E5CA21CA28EB5DC3CB616763CB5DC75
:1075400095D86E1C62EF85DC7C0AB34C8B7C581599
:10755000A27CF9DC9C623BE08E8E8E6AA09C154E6C
:1075600071AC3C66CF7CF659A471AC3CF687FC76D6
:107570007667B05DD4EDDC55A455ACB029DCCC37D2
:1075800001D068B02839CCC1CC5DAC7CEAC9DC1C28
:10759000AA7CA6FC289C107C16FC369616BC364BA2
:1075A00068E5D86221D97883385C507CF5DC369F59
:1075B000FC1C1050285C3DDC629C50D9D409DC2AAC
:1075C000A353163CB6F6C1C21C1050BC287C167CD6
:1075D000B6FC16763CB6BCD9D47940787CC461D868
:1075E000C8C1D409DC2A33BC76E3CD8CDD40213E12
:1075F00079D878BC06BCA6FC85D8614009BA680E6B
:10760000BA3C5CA2BC9C9BB813680EBA5CA2EE5C50
:10761000A2539C025A3CA2027CA23C607C06FCA6BF
:1076200016060E8E865C02A2A21F06EB56CC3B65A8
:10763000DCA67CE8FC70380E29AE654465DC70AED3
:10764000F0E30E5CA29CA25DDCA65C5DDCA01CE00D
:107650001C727CA695D8722F267C26CBA059A6FC3E
:10766000EECE1DAC0ECE7C1DACAEF0C65670AEF0AC
:10767000CE60E00E8E9CA27CA21FFCEB5CE2EE02D0
:10768000EE9CE0167CB6FC600EBC5C028DDB3C1C04
:10769000A25CA29CA286A665DC8EAE145F7C1CA6B2
:1076A000A626AAFC0A1C7BB5DC3C02BC4255A4F809
:1076B0007CA63CE8F8FC8EB68E8E861CAA7CE88DF3
:1076C000D8F87C1DAC65DC7DDCF8FC7659A7267CFF
:1076D000E8F87C81DCBCE85B3C163C16234E318E1E
:1076E0001C7C6A763C769C7C168686621F06EBBC08
:1076F000167CB681DC7C16FC56FC9C0E8E86621FC6
:1077000006EBBC0646BC16063C267C19DC8DD8B8B8
:107710000E1DACAE7C7DDCB81C7C6AEAA03CA9DC0A
:107720007C9DDCA86301D878603C36167C9616E018
:107730003C16FCB6B3C9DC3C3616BC9301D838BC49
:107740008DC40A7C8A0A7CE05C02EEDCA2E05C026A
:107750008ED4D30E4670F8FCE01DAC85384D400D3C
:1077600040A18863EE7841D8EE6544F055A4789C3A
:10777000FB55A4B8DBE5A0C80E301070B8BC8B3C3C
:1077800055A4AE685B5E55A4AEA82BEE1BA0BE60F0
:10779000E08EAEA6A26026EB1C2A068686601C0A36
:1077A000E0067CD306FCBBAEA6A626A6E056703843
:1077B0000E5E60F6631C1076333656F6333C3E1B85
:1077C000B63C3EE05DACE67A3C6AE7FCAA7C0E463D
:1077D00070AE680A2A6AAA7677F663567038C8F6D9
:1077E00033A0B660F660C4E00E4E5C22E0000000FC
:1077F000000000000000000000000000A61A0000C9
:10780000B21A0000B81A0000C41A0000CA1A000018
:10781000D61A00008C1A0000A01A00005A1D0000A1
:107820004A1D00003A1D0000341D0000221D00000A
:10783000101D0000FC1C0000EA1C0000D81C000009
:10784000C81C0000A81C0000861C0000761C00005C
:10785000541C0000341C0000161C0000F61B000025
:10786000D41B0000B41B0000921B0000E01A0000B3
:10787000DC1A00008C1B0000861B0000761B000039
:10788000561B0000441B0000301B0000221B0000A0
:10789000141B0000061B0000681D0000622300008E
:1078A000742300008623000098230000AA23000010
:1078B000C823000062230000E223000062230000CE
:1078C00062230000F4230000622300006223000012
:1078D00062230000FC230000042400002E2400008A
:1078E0006623000066230000662300006623000074
:1078F0006623000066230000662300006623000064
:107900006623000066230000662300008424000034
:107910006623000066230000662300006623000043
:107920006623000066230000662300006623000033
:10793000662300007C24000066230000AA240000C7
:10794000662300006623000066230000A2240000D6
:107950006623000066230000662300006623000003
:1079600066230000662300006623000066230000F3
:10797000662300009A240000662300009024000083
:10798000662300006623000066230000FA2400003E
:1079900066230000662300006623000066230000C3
:1079A00066230000662300006623000066230000B3
:1079B00066230000F224000066230000E824000093
:1079C000662300006623000066230000E024000018
:1079D0006623000066230000662300006623000083
:1079E0006623000066230000662300006623000073
:1079F0006623000066230000662300006623000063
:107A0000662300006623000066230000D8240000DF
:107A10006623000066230000662300006623000042
:107A20006623000066230000662300006623000032
:107A300066230000D02400006623000066230000B7
:107A4000662300006623000066230000C8240000AF
:107A50006623000066230000662300006623000002
:107A600066230000662300006623000066230000F2
:107A700066230000C024000066230000D425000017
:107A8000662300006623000066230000CC2500006A
:107A900066230000662300006623000066230000C2
:107AA00066230000662300006623000066230000B2
:107AB00066230000C4250000662300006623000042
:107AC0006623000066230000662300006623000092
:107AD0006623000066230000662300006623000082
:107AE0006623000066230000662300006623000072
:107AF000662300006623000066230000A82500001E
:107B00006623000066230000662300006623000051
:107B10006623000066230000662300006623000041
:107B20006623000066230000662300006623000031
:107B30006623000066230000662300009E250000E7
:107B400066230000662300006623000088250000ED
:107B50006623000066230000662300006623000001
:107B600066230000662300006623000066230000F1
:107B70006623000066230000662300007E250000C7
:107B800066230000662300006623000066230000D1
:107B900066230000662300006623000066230000C1
:107BA00066230000662300006623000066230000B1
:107BB0006623000066230000662300006E25000097
:107BC000662300006623000066230000662500008F
:107BD0006623000066230000662300006623000081
:107BE0006623000066230000662300006623000071
:107BF000662300006623000066230000562500006F
:107C00006623000066230000662300004E25000066
:107C10006623000066230000662300006623000040
:107C20006623000066230000662300006623000030
:107C3000662300004625000066230000382500006A
:107C40006623000066230000662300003025000044
:107C50006623000066230000662300006623000000
:107C600066230000662300006623000066230000F0
:107C7000662300002825000066230000022500007E
:107C800066230000662300006623000054240000E1
:107C900066230000662300006623000066230000C0
:107CA000DC2500002E2400004C2400006623000088
:107CB000642400005C240000322400001224000030
:107CC0000304050A08060BFF0209070D010C00FF5B
:107CD000202020205F5F7C002C0044697370206F9F
:107CE00066660D0A0055534552004600470042455E
:107CF00047494E0052414400442E4D590043005024
:107D000052474D0055534552202020006620200048
:107D100067202000424547494E2020202020005265
:107D2000414420202000442E4D5920202000432093
:037D300020200010
:107D3300103B000000000000E10C0000283B0000A5
:107D43002D3B00002B3B0000FF000000310600002C
:107D5300373B0000413B0000CF3A00000000000029
:107D630005040000533B00002D3B00005F3B000077
:107D73000000000029050000613B00002D3B0000CE
:107D83006D3B000000000000910600006F3B000007
:107D93002D3B00000F000000F4010000040103016B
:107DA3000201010411040F04170416011801000055
:107DB300047D00000C7D0000107D0000147D000098
:107DC300EC7C00001F7D0000267D00002E7D00005E
:107DD300FF7C000000171B243E4253697505020512
:107DE3000804080B0804040501050409080904062E
:107DF300080702060204020601060407010308033A
:107E0300040C080D020C0203020C010C040D010DFD
:107E1300080D0408020808070802020704080108FD
:107E230004090209010A080B020A0201080A010AED
:107E3300040B0102080204100811021002110810B9
:107E43000110041101120212011302130812080F88
:107E53000812041301130414021401150215081463
:107E63000817081404150115041702170119081A35
:107E73000219021602190119041A01160816041B25
:107E8300021B081A0818021A041B011B04180818FD
:107E9300040B04202020202020202020200000008C
:107EA30001000000E57C0000EA7C0000EC7C00009F
:107EB300EE7C0000EC7C0000F47C0000F87C000009
:087EC300FD7C0000FF7C0000C3
:040000030000323196
:00000001FF
